:020000040800F2
:10000000687600202903000831480008E54300080D
:100010002D480008CD0600080181000800000000FE
:10002000000000000000000000000000690200085D
:100030004B09000800000000C50200082B4D000815
:100040004303000843030008430300084303000878
:100050004303000843030008430300084303000868
:100060004303000843030008430300084303000858
:100070000108000843030008430300084303000885
:100080004303000843030008430300084303000838
:10009000D106000843030008430300084303000897
:1000A0004303000843030008430300084303000818
:1000B0004303000843030008430300084303000808
:1000C00043030008430300084303000843030008F8
:1000D000430300089558000843030008A55800088A
:1000E00043030008430300084303000843030008D8
:1000F00043030008430300084303000843030008C8
:1001000043030008430300084303000843030008B7
:1001100043030008430300084303000843030008A7
:1001200043030008110800082108000843030008E1
:100130004303000843030008430300084303000887
:1001400043030008E106000843030008354800089F
:10015000430300083108000843030008B9580008A9
:100160004303000843030008430300084303000857
:100170004303000843030008430300080000000095
:10018000430300084303000800F002F800F05CF8A5
:100190000AA090E8000C82448344AAF10107DA45E2
:1001A00001D100F051F8AFF2090EBAE80F0013F0D8
:1001B000010F18BFFB1A43F0010318472CB70000CA
:1001C0004CB700000A444FF0000C10F8013B13F04C
:1001D000070408BF10F8014B1D1108BF10F8015BA0
:1001E000641E05D010F8016B641E01F8016BF9D193
:1001F00013F0080F1EBF10F8014BAD1C0C1B09D1EA
:100200006D1E58BF01F801CBFAD505E014F8016B5B
:1002100001F8016B6D1EF9D59142D6D370470000ED
:100220000023002400250026103A28BF78C1FBD8FF
:10023000520728BF30C148BF0B6070471FB50BF095
:1002400043F81FBD10B510BD00F0D4F91146FFF7FB
:10025000F5FF08F08DFA00F0F2F903B4FFF7F2FFB2
:1002600003BC00F0F5F900002C4B19680868B0E8F1
:10027000F04F80F30988BFF36F8F4FF0000080F3D9
:10028000118870470000000008480068006880F38B
:1002900008884FF0000080F3148862B661B6BFF39F
:1002A0004F8FBFF36F8F00DF00BF00BF08ED00E08E
:1002B000DFF80C00016841F470010160704700BF75
:1002C00088ED00E0EFF30980BFF36F8F134B1A68DE
:1002D0001EF0100F08BF20ED108A20E9F04F1060CB
:1002E00009B44FF0500080F31188BFF34F8FBFF374
:1002F0006F8F09F041FE4FF0000080F3118809BCB8
:1003000019680868B0E8F04F1EF0100F08BFB0EC95
:10031000108A80F30988BFF36F8F70478000002038
:10032000EFF30580704700000948804709480047FF
:10033000FEE7FEE7FEE7FEE7FEE7FEE7FEE7FEE795
:10034000FEE7FEE704480549054A064B70470000F2
:10035000F14D000889010008686E002068760020D1
:10036000687200206872002053EA020C00F0698075
:100370002DE9F04B4FF00006002B1FBFB3FA83F5B9
:1003800003FA05F424FA05F65E4012BF1643B2FAEA
:1003900082F502FA05F4C5F120051EBF22FA05FC1C
:1003A00044EA0C04203556EA044C4FEA144418BFC2
:1003B000641C4FF000084FF00009904271EB030CF1
:1003C00039D3002919BFB1FA81F701FA07F6B0FA5B
:1003D00080F700FA07F6C7F120071EBF20FA07FCD6
:1003E00046EA0C062037B6FBF4FCA7EB0507103FE6
:1003F00007F01F0BCBF120060CFA0BFB2CFA06F6CC
:1004000044BFB3460026202FA4BF5E464FF0000B2A
:100410005BEA060C08BF4FF0010B19EB0B09ABFBB5
:10042000027C48EB0608C01B06FB02CC0BFB03CC8E
:1004300071EB0C01C1E70B46024641464846BDE858
:10044000F08B13B54FF000004FF00001AFF30080C8
:10045000BDE81C407047032A40F2308010F0030CC6
:1004600000F0158011F8013BBCF1020F624498BF07
:1004700011F801CB00F8013B38BF11F8013BA2F1A4
:10048000040298BF00F801CB38BF00F8013B11F01F
:10049000030300F05780083AC0F0088051F8043B8D
:1004A000083A51F804CBA0E80810F5E7121D5CBF2C
:1004B00051F8043B40F8043BAFF30080D20724BF5F
:1004C00011F8013B11F801CB48BF11F8012B24BFF3
:1004D00000F8013B00F801CB48BF00F8012B704742
:1004E00002F0FF0343EA032242EA024200F05EB850
:1004F0004FF0000200B5134694469646203922BFBD
:10050000A0E80C50A0E80C50B1F12001BFF4F7AF07
:10051000090728BFA0E80C5048BF0CC05DF804EBE9
:10052000890028BF40F8042B08BF704748BF20F857
:10053000022B11F0804F18BF00F8012B7047704755
:100540007047704710B5203AC0F00B80B1E81850E2
:10055000203AA0E81850B1E81850A0E81850BFF4AD
:10056000F5AF5FEA027C24BFB1E81850A0E818504C
:1005700044BF18C918C0BDE810405FEA827C24BFA0
:1005800051F8043B40F8043B08BF7047D20728BF2E
:1005900031F8023B48BF11F8012B28BF20F8023B7D
:1005A00048BF00F8012B70474FF000020429C0F04B
:1005B000128010F0030C3FF49DAFCCF1040CBCF1A1
:1005C000020F18BF00F8012BA8BF20F8022BA1EBE7
:1005D0000C01FFF78FBF5FEAC17C24BF00F8012B3D
:1005E00000F8012B48BF00F8012B70470048704706
:1005F000086E00207546FFF7F9FFAE460500694614
:10060000534620F00700854618B020B5FFF79AFE44
:10061000BDE820404FF000064FF000074FF0000803
:100620004FF0000B21F00701AC46ACE8C009ACE884
:10063000C009ACE8C009ACE8C0098D46704710B5E8
:100640000446AFF300802046BDE81040FFF705BE2A
:1006500001491820ABBEFEE72600020070470000EB
:1006600010B5034612B96FF0010010BD03EB830013
:1006700000EBC300034C04EB800040F82120002075
:10068000F3E70000406A002038B50446204604F035
:1006900097FE05462068006800F01000102811D170
:1006A00000BF00200090206800680090206840682B
:1006B000009000BF00BF05EBC501034A02EB8101BA
:1006C000086A804738BD0000A86A002000BFFEE726
:1006D00010B5024800F078FD10BD00000C020020AB
:1006E00010B5024800F070FD10BD0000340200207B
:1006F0000146074A0868904201D101207047054A27
:100700000868904201D10020F8E70320F6E70000D6
:1007100000680040006400402DE9F84304460D469F
:1007200016461F46DDF820804FF400700D49086022
:1007300000208860C86008200861200A0A49087003
:100740004C70280A8870CD70300A08714E71380AD2
:100750008871CF716B460A460249404600F015FB8E
:10076000BDE8F883E46B0020A00100200346042BC1
:1007700015D007DC7BB1012B0ED0022B0DD0032B43
:1007800012D10BE0202B0BD0212B0AD0222B09D029
:10079000232B09D107E008E007E006E005E004E0CC
:1007A00003E002E001E000E000BF00BF002070476E
:1007B0000020704710B500220449054805F01FFBD2
:1007C0000449034805F00CFB002010BD681200200E
:1007D0008C050020680A002070B504460D462146AD
:1007E000034805F0FDFA024805F0C6FA002070BD86
:1007F0008C05002010B503460C460021084610BDAC
:1008000010B5024801F072F910BD00006C04002020
:1008100010B5024801F06AF910BD0000CC040020B8
:1008200010B5024801F062F910BD00000C04002070
:1008300010B5024801F05AF910BD00002C05002047
:100840000146087810381823B0FBF3F20848805CA2
:10085000C865032A05D908686FF30900001D88657B
:1008600003E008686FF309008865886D7047000031
:10087000F8B20008014600208A6A8B69CBB932B110
:10088000012A0DD0022A03D0032A10D10EE000BFA6
:10089000CB6A03F08073B3F1807F00D1012007E0C1
:1008A000CB6AB3F1C07F00D1012001E000E000BFBE
:1008B00034E08B69B3F5005F1AD132B1012A07D059
:1008C000022A03D0032A11D10AE000BF01200EE062
:1008D000CB6A03F08073B3F1807F00D1012006E082
:1008E000CB6AB3F1C07F00D1012000E000BF15E06A
:1008F00032B1012A05D0022A04D0032A0CD103E028
:1009000000BF00BF012008E0CB6A03F08073B3F1A1
:10091000807F00D1012000E000BF00BF704730B5EC
:100920000468246824F4802405682C6004686360EB
:100930008468402C04D10468A2600468E16003E08C
:100940000468A1600468E26030BD704710B5064BD2
:10095000064A0021064800F06DFB042105480068A6
:1009600008F026F810BD0000A8010020FC6B002054
:100970000C020020B001002072B600BFFEE70000AC
:1009800010B500205BE000EB4001314A02EB411161
:100990000880012100EB40022D4B03EB42125180F5
:1009A00000EB400203EB42129180002100EB400279
:1009B00003EB4212916000EB400203EB4212D16064
:1009C0009FED240A00EB40011A4602EB411181ED34
:1009D000040A9FED200A00EB400102EB411181ED7A
:1009E000050A9FED1C0A00EB400102EB411181ED6D
:1009F000060A9FED180A00EB400102EB411181ED60
:100A0000070A9FED140A00EB400102EB411181ED52
:100A1000080A002100EB400203EB42125162FE2162
:100A200000EB400203EB421282F82810EE2200EBAA
:100A3000400103EB411181F82920411CC8B2022872
:100A4000A1DB054A0121054803F0E4FB10BD0000CD
:100A5000186C002000000000959800089403002006
:100A60002DE9F0412DED048B05464FF0FF36A878B7
:100A700000F00F0606EB4600304901EB401410224F
:100A8000294604F13900FFF7E6FCA87800096080E8
:100A90000120A0800020A060E878297940EA0120A8
:100AA00000B208EE100AB8EEC80A84ED060A94ED0A
:100AB000060ADFED230A80EE201A84ED061A687913
:100AC000A97940EA012000B208EE900AB8EEE80ADF
:100AD00084ED070A94ED070ADFED1A0A20EE200ADA
:100AE000DFED190A80EE201A84ED071AA87A0006B5
:100AF000697A40EA0140297A40EA0120E97908430D
:100B000009EE100AB8EEC90A84ED080A94ED080A45
:100B1000DFED0C0A20EE200ADFED0C0A80EE201A31
:100B200084ED081AE87A47B2E760287B00F00700F6
:100B3000A060BDEC048BBDE8F0810000186C0020C3
:100B400000008043E40FC9405C8FCA445C8F4A4870
:100B50002DE9F0472DED068B81460E461746B0EE87
:100B6000408AF0EE608AB0EE419AF0EE619AB0EE03
:100B700042AA06EB4600634901EB4014012F09D15C
:100B8000112204F12801484603F0DEFBBDEC068B80
:100B9000BDE8F087FE2084F84C00EE214D20015581
:100BA00020784E21095D60F303014E200155A078A5
:100BB0004E21095D60F306114E200155005D20F0C5
:100BC00080014E2001559FED500A28EE000ABDEE2F
:100BD000C00A10EE100A01B2502001539FED4A0ADC
:100BE00029EE000ADFED490A20EE200ADFED480A6F
:100BF00080EE201ABDEEC10A10EE100A01B2A4F870
:100C000052109FED440A28EE800ADFED400A20EEE4
:100C1000200ADFED3F0A80EE201ABDEEC10A84ED06
:100C2000150A9FED3D0A29EE800ABCEEC00A10EEBF
:100C3000100AA4F858009FED380A2AEE000ABCEE0C
:100C4000C00A10EE100AA4F85A0004F14E0898F8F1
:100C500000102A2001555020015D2B200155502005
:100C6000005BC0F307212C20015594F852102D2071
:100C70000155B4F85200C0F307212E20015594F815
:100C800054102F200155B4F85400C0F30721302030
:100C90000155606DC0F3074131200155606D010EB3
:100CA0003220015594F8581033200155B4F85800FB
:100CB000010A3420015594F85A1035200155B4F832
:100CC0005A00010A362001550F2104F1280007F0CF
:100CD00045FC054637200555290A382001551122C3
:100CE00004F12801484603F02FFB0C4908706420EA
:100CF00001F0DCF810220A49484603F075FA00BFFB
:100D000044E70000186C0020000080435C8FCA405C
:100D1000E40FC940000000470000A044B5010020D6
:100D2000D86C002000487047B801002070B50A4810
:100D30000468001D0568001D0668344454B108228B
:100D40000649204603F050FB04220449103128468E
:100D500003F04AFB70BD0000107AFF1F4200002024
:100D600010B5024692F82030012B01D0022B06D19B
:100D700010684069084314686061002010BD506A23
:100D800040F4802050620120F8E7F0B504460D469B
:100D90001E4694F8207020688368A86800B900E0B7
:100DA00000BF012F01D0022F7DD103F0806030B948
:100DB00003F0006018B903F0805000287ED0C3F320
:100DC0000161012088403060A86860B9B5F800C0B2
:100DD000E86840EA4C5C206800F5C07000EB011048
:100DE000C0F800C00FE0D5E901C040EACC00D5F85A
:100DF0000CC040EA0C00D4F800C00CF5C07C0CEB31
:100E0000011CCCF80000D5F810C0206800F5C070B7
:100E100000EB0110C0F804C0287D01280ED1206825
:100E200000F5C07000EB0110406840F4807C206841
:100E300000F5C07000EB0110C0F804C0D0790006C6
:100E400092F806C040EA0C4092F805C040EA0C2037
:100E500092F804C040EA0C00D4F800C00CF5C07C45
:100E60000CEB011CCCF80C00D078000692F802C004
:100E700040EA0C4092F801C040EA0C2092F800C011
:100E800040EA0C00D4F800C00CF5C07C0CEB011C4F
:100E9000CCF80800206800F5C07000EB0110006875
:100EA00040F0010C01E00FE008E0206800F5C070A0
:100EB00000EB0110C0F800C00020F0BD606A40F4F3
:100EC000001060620120F8E7606A40F480206062F0
:100ED0000120F2E7F0B504460A46216894F8205054
:100EE000012D01D0022D7ED1424901F50071086823
:100EF00040F001000860086820F47C500860086831
:100F0000566A40EA06200860107D00F01F060120A6
:100F100000FA06F3C8699843C861A1F50071D06969
:100F2000C8B9D1F80C029843C1F80C02908880B27D
:100F3000968940EA064601F51070576940F8376017
:100F4000108880B2168940EA064601F5107057698C
:100F500000EBC7004660D069012819D1D1F80C0216
:100F60001843C1F80C02908880B2168840EA064601
:100F700001F51070576940F83760908980B2168982
:100F800040EA064601F51070576900EBC70046605D
:100F9000906928B9D1F804029843C1F8040204E02A
:100FA000D1F804021843C1F80402106928B9D1F835
:100FB00014029843C1F8140204E0D1F81402184353
:100FC000C1F81402106A012804D1D1F81C02184398
:100FD000C1F81C02D1F8000220F00100C1F80002A3
:100FE0000020F0BDFFE7606A40F4802060620120CD
:100FF000F7E700000064004070B505462846FFF79B
:1010000077FB0446032C11D004EB840000EBC400F2
:10101000074901EB8000006B40B104EB840101EB58
:10102000C401034A02EB8101086B804770BD0000D8
:10103000406A002070B5044694F82050012D01D07C
:10104000022D7DD151B92068C06800F0030080B93D
:10105000606A40F400106062012070BD2068006981
:1010600000F0030028B9606A40F4001060620120BB
:10107000F3E7206800F5D87000EB0110006800F07D
:1010800004009060906840B9206800F5D87000EBCB
:1010900001100068400D106007E0206800F5D8706E
:1010A00000EB01100068C0085060206800F5D8709F
:1010B00000EB0110006800F00200D060206800F52D
:1010C000D87000EB0110406800F00F00082802D330
:1010D0000820106108E0206800F5D87000EB0110CE
:1010E000406800F00F001061206800F5D87000EB38
:1010F0000110406800F47F40000A9061206800F50C
:10110000D87000EB01104068000C5061206800F5B9
:10111000D87000EB011080681870206800F5D87056
:1011200000EB0110806800F47F40000A58702068CE
:1011300000F5D87000EB0110806800F47F0000E03B
:101140003CE0000C9870206800F5D87000EB0110AE
:101150008068000ED870206800F5D87000EB011090
:10116000C0681871206800F5D87000EB0110C068E5
:1011700000F47F40000A5871206800F5D87000EB39
:101180000110C06800F47F00000C9871206800F521
:10119000D87000EB0110C068000ED87131B920681A
:1011A000C06840F020002668F06005E02068006913
:1011B00040F020002668306100204EE7606A40F46D
:1011C00080206062012048E72DE9F05F0446002599
:1011D000206846692068D0F80490206887682068F5
:1011E000D0F80CA02068D0F810B02068D0F8188093
:1011F00006F00100002855D007F00100C0B1012021
:101200002168886007F0020018B1204600F052FB08
:101210000EE007F0040010B145F4006508E007F0A7
:10122000080010B145F4805502E0204600F024FB90
:1012300007F48070C8B14FF480702168886007F4AB
:10124000007018B1204600F06FFB0EE007F48060DC
:1012500010B145F4005508E007F4006010B145F402
:10126000804502E0204600F041FB07F48030C8B121
:101270004FF480302168886007F4003018B12046B0
:1012800000F08EFB0EE007F4802010B145F400451D
:1012900008E007F4002010B145F4803502E0204654
:1012A00000F060FB06F0080038B10AF0100020B131
:1012B00045F4007510202168C86006F0040040B1B4
:1012C0000AF0080028B108202168C860204600F014
:1012D0000DFA06F0020038B12068C06800F0030083
:1012E00010B1204600F020FA06F0400038B10BF0B3
:1012F000100020B145F4806510202168086106F0D7
:10130000200040B10BF0080028B1082021680861D6
:10131000204600F027FA06F0100038B12068006976
:1013200000F0030010B1204600F03AFA06F4003055
:1013300040B109F0100028B1102021684860204613
:1013400000F04CFA06F4803040B109F0080028B1F2
:10135000082021684860204600F040FB06F4004069
:1013600088B309F0040078B306F4807020B108F067
:10137000010008B145F0010506F4007020B108F045
:10138000020008B145F0020506F4806020B108F0C3
:10139000040008B145F0040506F40060A0B108F0AF
:1013A000700088B108F07000402817D006DC1028C3
:1013B0000BD020280CD0302819D10CE0502810D0A8
:1013C000602814D110E01DE019E045F008050FE099
:1013D00045F010050CE045F0200509E045F040051A
:1013E00006E045F0800503E045F4807500E000BFAD
:1013F00000BF2068806920F07000216888610420A7
:10140000216848602DB1606A284360622046FFF77A
:10141000F3FDBDE8F09F70B504460CB9012070BD26
:1014200094F8200010B9204600F0B0F82068006859
:1014300040F001002168086000F04CFE05460DE018
:1014400000F048FE401B0A2808D9606A40F40030CA
:101450006062052084F820000120E0E720684068F1
:1014600000F001000028EBD02068006820F00200A6
:101470002168086000F02EFE05460DE000F02AFE0F
:10148000401B0A2808D9606A40F4003060620520D9
:1014900084F820000120C2E72068406800F00200C4
:1014A0000028EBD1207E012806D12068006840F09A
:1014B00080002168086005E02068006820F0800056
:1014C00021680860607E012806D12068006840F02D
:1014D00040002168086005E02068006820F04000B6
:1014E00021680860A07E012806D12068006840F0CD
:1014F00020002168086005E02068006820F02000D6
:1015000021680860E07E012806D12068006820F08C
:1015100010002168086005E02068006840F01000B5
:1015200021680860207F012806D12068006840F00B
:1015300008002168086005E02068006820F00800C5
:1015400021680860607F012806D12068006840F0AB
:1015500004002168086005E02068006820F00400AD
:1015600021680860D4E902010843216908436169E0
:1015700008436168491E08432168C8610020606211
:10158000012084F82000002049E7000010B586B053
:101590000446142101A8FEF7ABFF4E49206888429B
:1015A00041D14D480068401C4B490860084600681E
:1015B00001280FD100BF002000904848006840F08B
:1015C0000070464908600846006800F0007000900E
:1015D00000BF00BF00BF00200090404810380068E6
:1015E00040F008003D49103908600846006800F0E6
:1015F0000800009000BF00BF03200190022002906D
:1016000000200390032004900920059001A934488C
:1016100000F060FC00220521142000F0EFFD1420F2
:1016200000F0D8FD54E02F492068884250D100BF17
:10163000002000902948006840F080602749086039
:101640000846006800F08060009000BF00BF22489C
:101650000068401C204908600846006801280FD136
:1016600000BF002000901D48006840F000701B493A
:1016700008600846006800F00070009000BF00BFDE
:1016800000BF0020009015481038006840F00200AC
:101690001249103908600846006800F00200009006
:1016A00000BF00BF60200190022002900020039044
:1016B000032004900920059001A90B4800F00AFCC2
:1016C00000220521412000F099FD412000F082FD1B
:1016D00006B010BD00640040080000204038024001
:1016E000000C0240006800400004024070B505464E
:1016F0002846FEF7FDFF0446032C11D004EB8400BE
:1017000000EBC400074901EB8000C06940B104EB65
:10171000840101EBC401034A02EB8101C8698047DF
:1017200070BD0000406A002070B505462846FEF7EF
:10173000DFFF0446032C11D004EB840000EBC4004F
:10174000074901EB8000806940B104EB840101EBA3
:10175000C401034A02EB81018869804770BD000023
:10176000406A002070B505462846FEF7C1FF0446D2
:10177000032C11D004EB840000EBC400074901EBFB
:101780008000406A40B104EB840101EBC401034ACC
:1017900002EB8101486A804770BD0000406A00206A
:1017A00070B505462846FEF7A3FF0446032C11D06A
:1017B00004EB840000EBC400074901EB8000006AE1
:1017C00040B104EB840101EBC401034A02EB810147
:1017D000086A804770BD0000406A002070B5054669
:1017E0002846FEF785FF0446032C11D004EB840045
:1017F00000EBC400074901EB8000806A40B104EBB4
:10180000840101EBC401034A02EB8101886A80472D
:1018100070BD0000406A002070B5044694F82000B6
:10182000012822D1022084F820002068006820F0DE
:1018300001002168086000F04DFC05460DE000F055
:1018400049FC401B0A2808D9606A40F400306062F5
:10185000052084F82000012070BD2068406800F059
:1018600001000028EBD16062F6E7606A40F40020D6
:1018700060620120F0E7000070B505462846FEF7DB
:1018800037FF0446032C11D004EB840000EBC400A6
:10189000074901EB8000C06840B104EB840101EB13
:1018A000C401034A02EB8101C868804770BD000093
:1018B000406A002070B505462846FEF719FF044629
:1018C000032C0FD004EB840000EBC400064951F850
:1018D000200038B104EB840101EBC401024A52F844
:1018E0002100804770BD0000406A002070B50546A9
:1018F0002846FEF7FDFE0446032C11D004EB8400BD
:1019000000EBC400074901EB8000006940B104EB23
:10191000840101EBC401034A02EB8101086980479D
:1019200070BD0000406A002070B505462846FEF7ED
:10193000DFFE0446032C11D004EB840000EBC4004E
:10194000074901EB8000406840B104EB840101EBE2
:10195000C401034A02EB81014868804770BD000062
:10196000406A002070B505462846FEF7C1FE0446D1
:10197000032C11D004EB840000EBC400074901EBF9
:101980008000406940B104EB840101EBC401034ACB
:1019900002EB81014869804770BD0000406A002069
:1019A00070B505462846FEF7A3FE0446032C11D069
:1019B00004EB840000EBC400074901EB8000806861
:1019C00040B104EB840101EBC401034A02EB810145
:1019D0008868804770BD0000406A002070B50546E9
:1019E0002846FEF785FE0446032C11D004EB840044
:1019F00000EBC400074901EB8000C06A40B104EB72
:101A0000840101EBC401034A02EB8101C86A8047EB
:101A100070BD0000406A002070B50446A56D00F05E
:101A200059FB064694F83500022808D080206065EE
:101A300000BF002084F8340000BF012070BD206882
:101A4000006820F01600216808602068406920F0D6
:101A5000800021684861206C08B9A06C28B120681A
:101A6000006820F00800216808602068006820F005
:101A700001002168086010E000F02CFB801B0528A5
:101A80000BD920206065032084F8350000BF0020BA
:101A900084F8340000BF0320D0E72068006800F01D
:101AA00001000028E8D194F85C103F208840A8602D
:101AB000012084F8350000BF002084F8340000BF06
:101AC00000BFBBE7014691F83500022803D0802013
:101AD000486501207047052081F8350008680068D6
:101AE00020F001000A6810600020F3E7F8B5044612
:101AF000002000908C4800684FF41651B0FBF1F7BD
:101B0000A56D2E6894F85C1008208840304098B18C
:101B10002068006800F0040070B12068006820F0C0
:101B200004002168086094F85C1008208840A860D0
:101B3000606D40F00100606594F85C100120884001
:101B4000304068B12068406900F0800040B194F8EE
:101B50005C1001208840A860606D40F00200606564
:101B600094F85C1004208840304068B12068006818
:101B700000F0020040B194F85C1004208840A86096
:101B8000606D40F00400606594F85C10102088409F
:101B9000304078B32068006800F0080050B394F833
:101BA0005C1010208840A8602068006800F4802045
:101BB00080B12068006800F4002028B9206CC8B10A
:101BC0002046216C884715E0A06C98B12046A16C96
:101BD00088470FE02068006800F4807028B920680A
:101BE000006820F0080021680860206C10B12046D1
:101BF000216C884794F85C102020884030400028F1
:101C000065D02068006800F0100000285FD094F8CC
:101C10005C1020208840A86094F83500052828D161
:101C20002068006820F0160021680860206840697C
:101C300020F0800021684861206C08B9A06C28B1B0
:101C40002068006820F008002168086094F85C10A3
:101C50003F208840A860012084F8350000BF0020A4
:101C600084F8340000BF206D10B12046216D8847F4
:101C7000F8BD2068006800F4802080B1206800680A
:101C800000F4002028B9606C10B12046616C8847D0
:101C90001DE0E06BD8B12046E16B884717E0206873
:101CA000006800F4807068B92068006820F01000B7
:101CB00021680860012084F8350000BF002084F806
:101CC000340000BFE06B10B12046E16B8847606DC7
:101CD00038B3606D00F00100F0B1052084F83500E4
:101CE0002068006820F001002168086000BF0098AB
:101CF000401C0090B84200D905E02068006800F060
:101D000001000028F3D100BF012084F8350000BF96
:101D1000002084F8340000BFE06C10B12046E16C74
:101D2000884700BFA4E700007C0000202DE9F041B7
:101D30000446002500F0CEF9074614B90120BDE89D
:101D4000F081606A00B100BF022084F8350000BF56
:101D5000002084F8340000BF2068006820F00100F3
:101D6000216808600AE000F0B5F9C01B052805D914
:101D700020206065032084F83500E0E720680068D3
:101D800000F001000028EED12068056821480540D8
:101D9000D4E901010843E168084321690843616906
:101DA0000843A1690843E1690843216A08430543E0
:101DB000606A042803D1D4E90B0108430543206875
:101DC00005602068456925F00705606A0543606A7B
:101DD00004280DD1A06A0543E06A48B12046FEF709
:101DE00049FD28B140206065012084F83500A6E750
:101DF000206845612046FEF723FD064694F85C10F6
:101E00003F208840B06000206065012084F83500E4
:101E1000002094E73F8010F02DE9F04704460D467E
:101E200016461F464FF00008D4F8589000BF94F8AB
:101E30003400012802D10220BDE8F087012084F897
:101E4000340000BF94F83500012825D1022084F821
:101E50003500002060653B46324629462046FEF7A5
:101E60005EFD94F85C103F208840C9F808002068A7
:101E7000006840F0160021680860206C28B12068D6
:101E8000006840F00800216808602068006840F0A1
:101E900001002168086006E000BF002084F83400DB
:101EA00000BF4FF002084046C6E7000070B5044688
:101EB00000F010F906462546681C10B10448007869
:101EC000054400BF00F006F9801BA842FAD370BD9C
:101ED00078000020F8B502460B46002500240020BB
:101EE0000021D6E0012606FA01F51E6806EA05047F
:101EF000AC4274D11E7906F00306012E04D01E797F
:101F000006F00306022E13D190684F000326BE4050
:101F1000B0434F00DE68BE403043906050680126F9
:101F20008E40B0431E79C6F300168E403043506099
:101F30001E7906F00306032E09D0D0684F00032651
:101F4000BE40B0434F009E68BE403043D0601E7913
:101F500006F00306022E13D1CF0802F1200656F830
:101F600027004E07F70E0F26BE40B0434F07FF0E67
:101F70001E69BE403043CF0802F1200646F8270014
:101F800010684F000326BE40B0431E7906F00306DA
:101F90004F00BE40304310605E6806F44036002EAD
:101FA00076D000BF002600963C4E366846F4804648
:101FB0003A4F3E603E46366806F48046009600BFC3
:101FC00000BF374E8F0856F827008E07370F0F26B1
:101FD000BE40B043334EB24202D1002624E057E067
:101FE000314EB24201D101261EE0304EB24201D143
:101FF000022619E02E4EB24201D1032614E02D4EE6
:10200000B24201D104260FE02B4EB24201D1052687
:102010000AE02A4EB24201D1062605E0284EB2421D
:1020200001D1072600E008268F073F0FBE4030434E
:102030001B4E8F0846F82700224E3068A0435E688A
:1020400006F4801606B120431E4E3060361D3068FF
:10205000A0435E6806F4001606B12043194E361DF3
:102060003060184E361F3068A0435E6806F40036B4
:1020700006B12043134E361F3060361F3068A04330
:102080005E6806F4803606B120430E4E083E30608E
:10209000491C1029FFF426AFF8BD00004438024067
:1020A00008380140000002400004024000080240DD
:1020B000000C0240001002400014024000180240D0
:1020C000001C0240083C01400AB1816101E00B04A0
:1020D000836170470148006870470000700000206D
:1020E00003480068034909780844014908607047BB
:1020F000700000207800002010B50D48006840F402
:1021000000700B4908600846006840F48060086071
:102110000846006840F480700860032000F0ACF8C6
:102120000F2000F007F800F02BF8002010BD000091
:10213000003C024070B504460E4800784FF47A71B6
:10214000B1FBF0F00C490968B1FBF0F5284601F04D
:1021500007FB08B1012070BD102C07D200222146D8
:10216000501E00F04BF80548046001E00120F2E742
:102170000020F0E7780000207C00002074000020A0
:1021800008B500BF002000901148006840F480406E
:102190000F4908600846006800F48040009000BFC6
:1021A00000BF00BF00200090081F006840F0805072
:1021B000091F08600846006800F08050009000BFCA
:1021C00000BF00220F21901E00F018F808BD00008B
:1021D000443802400146084600280DDB00BF00BF1E
:1021E00000F01F0301229A4043099B0003F1E02302
:1021F000C3F8002100BF00BF00BF70472DE9F05FAA
:1022000080460D461646002705F0BCFF07463946B6
:102210002A46334601F00700C0F1070ABAF1040F5D
:1022200002D94FF0040A01E0C0F1070AD14600F1DB
:10223000040ABAF1070F02D24FF0000A01E0A0F140
:10224000030AD4464FF0010A0AFA09FAAAF1010A70
:102250000AEA020A0AFA0CFA4FF0010B0BFA0CFB1D
:10226000ABF1010B0BEA030B4AEA0B042146404693
:1022700005F090FFBDE8F09F00BF00F00702064B9D
:1022800019684FF6FF031940044B0B4343EA022140
:10229000014B196000BF70470CED00E00000FA052B
:1022A000704702461068416200207047F0B503464F
:1022B00015461868446A21B944EA05401E68B062B0
:1022C00019E01868806A04EB1044002208E01868DE
:1022D00000F5827050F8220004EB1044501CC2B28A
:1022E000481E9042F3D844EA0547186800F582700A
:1022F0004E1E40F826700020F0BD10B50446D4F8FC
:10230000E00404F072FA10BD70B504460D4605EB0A
:10231000C50304F1140101EB8301CA682946D4F80E
:10232000E00404F05DF970BD70B504460D4605EBA0
:10233000C50304F5157101EB8301CA682946D4F879
:10234000E00404F0D1F970BD10B50446D4F8E004FF
:1023500004F04EFA10BD2DE9F04104460D4605F09B
:102360008000802808D105F00F0000EBC00104F1C7
:10237000140000EB810607E005F00F0000EBC00140
:1023800004F5157000EB81063146206805F07AFCF3
:1023900007463846BDE8F08170B504460E4606F0A3
:1023A000800080280AD106F00F0000EBC00104F184
:1023B000140000EB81050120687009E006F00F00B1
:1023C00000EBC00104F5157000EB8105002068707A
:1023D00006F00F00287000BF94F89404012801D182
:1023E000022070BD012084F8940400BF29462068B3
:1023F00004F0D6FF00BF002084F8940400BF00BFA3
:10240000EFE770B504460E4606F00F0021798842CA
:1024100001D9012070BD06F0800080280AD106F0A5
:102420000F0000EBC00104F1140000EB8105012056
:10243000687009E006F00F0000EBC00104F51570AC
:1024400000EB8105002068700020A87006F00F00E6
:10245000287000BF94F89404012801D10220D9E724
:10246000012084F8940400BF2946206805F096F9FD
:1024700000BF002084F8940400BF00BFCAE70246F2
:1024800001F00F0000EBC00302F5157000EB8300B4
:10249000406970472DE9F04705460E4690461F46B5
:1024A0004FF0000906F0800080280AD106F00F00E6
:1024B00000EBC00105F1140000EB81040120607005
:1024C00009E006F00F0000EBC00105F5157000EB08
:1024D00081040020607006F00F002070C8F30A002D
:1024E000A0602771607808B120786083022F01D145
:1024F0000020607100BF95F89404012802D10220E9
:10250000BDE8F087012085F8940400BF21462868C3
:1025100004F05AFE00BF002085F8940400BF48462E
:10252000EEE72DE9F04105460E461746984606F0BF
:102530000F0000EBC00105F5157000EB8104E760AA
:10254000C4F8108000206061607006F00F002070F9
:10255000A879012800D1E761AA792146286805F009
:10256000B1F90020BDE8F08170B504460D4605F0D4
:102570000F002179884201D9012070BD05F080004B
:1025800080280AD105F00F0000EBC00104F114000F
:1025900000EB81060120707007E005EBC50104F532
:1025A000157000EB8106002070700120B07005F0FE
:1025B0000F00307000BF94F89404012801D102206C
:1025C000DBE7012084F8940400BF3146206805F061
:1025D0002CF905F00F0028B9A17904F29C4220687B
:1025E00005F0A4F800BF002084F8940400BF00BFE9
:1025F000C3E72DE9F04105460E461746984606F01A
:102600000F0000EBC00105F1140000EB8104E7604E
:10261000C4F81080002060610120607006F00F0097
:102620002070A879012800D1E761AA79214628689D
:1026300005F048F90020BDE8F0812DE9FE4F044681
:10264000D4F800B05E46206805F0FEFB002874D187
:10265000206805F038FC08B9BDE8FE8F40F6080098
:102660008059C0F30D20C4F8D404206805F02BFC79
:1026700000F00200022805D12068406900F0020045
:1026800021684861206805F01EFC00F01000102849
:1026900045D12068806920F0100021688861DBF84E
:1026A000209009F00F0000EBC00104F5157000EB5D
:1026B000810AC9F3434002281AD147F6F07009EAAB
:1026C000000030B3C9F30A125846DAF80C1005F0CE
:1026D000FFFBC9F30A11DAF80C000844CAF80C0031
:1026E000C9F30A11DAF814000844CAF8140010E01B
:1026F000C9F3434006280CD1082204F29C415846F5
:1027000005F0E6FBC9F30A11DAF814000844CAF828
:1027100014002068806940F01000216888612068FA
:1027200005F0D1FB00F40020B0F5002F7BD100258F
:10273000206805F098FB029072E0E1E2029800F058
:102740000100002868D0E9B2206805F0AFFB8046A0
:1027500008F0010048B1012106F5306000EB45109A
:1027600081602946204602F0A9F808F008000828F0
:1027700009D1082106F5306000EB4510816029463B
:10278000204602F069F808F01000102805D1102149
:1027900006F5306000EB4510816008F00200022869
:1027A00024D1DBF8140000F08000802807D140F627
:1027B0000400805940F4806140F60400815105EB2B
:1027C000C50104F5157000EB810A9AF80300012891
:1027D00006D100208AF80300E9B2204600F09BFAF7
:1027E000022106F5306000EB4510816008F0200002
:1027F000202805D1202106F5306000EB45108160CE
:1028000008F40050B0F5005F06D14FF4005106F512
:10281000306000EB451081606D1C0298400802900A
:10282000029800288AD1206805F04DFB00F4802032
:10283000B0F5802F7DD1206805F00BFB02900025BC
:102840009AE0029800F00100002873D0E9B22068F5
:1028500005F013FB804608F00100F0B305F00F010E
:1028600001208840019040F634008159019821EA06
:10287000000040F634018851012106F5106000EB9C
:1028800045108160A079012824D105EBC50104F130
:10289000140000EB810005EBC502C16804F11400CF
:1028A00000EB82008068014405EBC50204F11400CE
:1028B00000EB8200C1606DB905EBC50104F11400A5
:1028C00000EB8100006928B904F29C4201212068D4
:1028D00004F02CFFE9B2204600E001E0FFF714FD10
:1028E00008F00800082805D1082106F5106000EB63
:1028F0004510816008F01000102805D1102106F560
:10290000106000EB4510816008F04000402805D1C0
:10291000402106F5106000EB4510816008F00200D0
:1029200002281DD12946584605F051FA05EBC5018C
:1029300001E025E01CE004F1140000EB810A9AF8A4
:102940000300012806D100208AF80300E9B22046DE
:1029500000F0D8F9022106F5106000EB4510816007
:1029600008F08000802803D12946204602F048F86C
:102970006D1C029840080290029800287FF461AF15
:10298000206805F0A0FA00F00040B0F1004F1CD123
:1029900040F60400805920F0010140F60400815106
:1029A00094F8CC04012807D1002084F8CC0400213D
:1029B0002046FFF775FC02E0204600F0D1FA2068BF
:1029C000406900F0004021684861206805F07BFA0A
:1029D00000F40060B0F5006F0ED140F60800805999
:1029E00000F0010010B1204600F012FB20684069A1
:1029F00000F4006021684861206805F064FA00F482
:102A00008050B0F5805F7ED140F60400805920F000
:102A1000010140F6040081511021206805F0D7F92A
:102A2000002732E04FF67F3106F5106000EB4710CB
:102A3000816006F5106000EB4710006820F400117B
:102A400006F5106000EB471001604FF67F3106F588
:102A5000306000EB4710816006F5306000EB4710F6
:102A6000006820F4001106F5306000EB47100160AB
:102A700006F5306000EB4710006840F0006106F595
:102A8000306000EB471001607F1C2079B842C9D844
:102A900040F61C00805940F0011140F61C008151A5
:102AA000E07B70B1D6F8840840F00B01C6F88418BA
:102AB00040F64400805940F00B0140F6440081513B
:102AC0000FE040F61400805942F22B01084340F613
:102AD00014018851081F805940F00B014FF4016028
:102AE0008151D6F8000820F4FE60C6F80008A179EC
:102AF00004F29C42206804F019FE2068406900F44A
:102B00008050216800E000E04861206805F0DBF9B2
:102B100000F40050B0F5005F17D1206804F0BCFB52
:102B2000206805F07EF9E07100F04EFB0090E2793C
:102B30002068009905F04EFA204600F0F9F9206867
:102B4000406900F4005021684861206805F0BBF935
:102B500000F00800082808D1204600F008FA206894
:102B6000406900F0080021684861206805F0ABF971
:102B700000F08000802818D1DBF8180020F08000D9
:102B8000CBF8180001250DE005EBC50104F5157023
:102B900000EB8100C078012803D1E9B22046FFF79D
:102BA000DAFB6D1C2079A842EED8206805F08BF97D
:102BB00000F48010B0F5801F2DD1012522E006F52C
:102BC000106000EB4510D0F8009005EBC50104F152
:102BD000140000EB81000079012812D109F00040B7
:102BE000B0F1004F0DD1012105EBC50204F1140035
:102BF00000EB8200C170E8B240F080012046FFF790
:102C0000AAFB6D1C2079A842D9D82068406900F43D
:102C1000801021684861206805F055F900F4001023
:102C2000B0F5001F44D1012538E006F5306000EB17
:102C30004510D0F8009005EBC50104F5157000EBC8
:102C400081000079012828D109F00040B0F1004F3F
:102C500023D109F4803094F8D41401F001018842A2
:102C60001BD1012105EBC50204F5157000EB8200B4
:102C7000C170DBF8180040F08000CBF81800DBF8DA
:102C8000140000F0800040B940F60400805940F480
:102C9000007140F60400815103E06D1C2079A842C8
:102CA000C3D800BF2068406900F400102168486163
:102CB000206805F008F900F08040B0F1804F08D19D
:102CC0002046FFF71AFB2068406900F08040216829
:102CD0004861206805F0F7F800F0040004280FD1DF
:102CE0002068D0F8049009F00400042802D120469E
:102CF000FFF72AFB2068406840EA09002168486025
:102D000000BFA9E470B504460D462946D4F8E00496
:102D100003F0DAFD70BD70B504460D462946D4F8BF
:102D2000E00403F0F5FD70BDF8B504460CB90120D0
:102D3000F8BD266894F8950428B9002084F8940416
:102D4000204600F0A1F8032084F89504B6F1A04FC6
:102D500001D10021A171206804F0E0FC207C8DF8F5
:102D6000000094E80F0004F0ABFA20B1022084F8D0
:102D700095040120DCE70021206805F0D9F820B196
:102D8000022084F895040120D2E7002531E00121DA
:102D900005EBC50204F1140000EB8200417005EB65
:102DA000C50104F1140000F8215005EBC50100EB4A
:102DB00081004583002105EBC50204F1140000EBFE
:102DC0008200017105EBC50204F1140000EB8200E2
:102DD000816005EBC50204F1140000EB8200C160C4
:102DE00005EBC50204F1140000EB82000161681CD0
:102DF000C5B22079A842CADC00252AE0002105EBF3
:102E0000C50204F5157000EB8200417005EBC501A9
:102E100004F5157000F82150002105EBC50200EB08
:102E20008200017105EBC50204F5157000EB82000C
:102E3000816005EBC50204F5157000EB8200C160EE
:102E400005EBC50204F5157000EB82000161681CFA
:102E5000C5B22079A842D1DC207C8DF8000094E82E
:102E60000F0004F067FB20B1022084F895040120D4
:102E70005EE700206074012084F89504206804F067
:102E800047FB002054E7000010B586B0044614212B
:102E900001A8FDF72DFB2068B0F1A04F42D100BF83
:102EA000002000902048006840F001001E490860A2
:102EB0000846006800F00100009000BF00BF4FF41A
:102EC000C050019002200290002003900320049043
:102ED0000A20059001A91548FEF7FCFF00BF124823
:102EE000001D006840F080000F49091D086000BF08
:102EF000002000900C481430006840F480400A49DB
:102F0000143108600846006800F48040009000BF5B
:102F100000BF00BF002205214320FFF76FF94320C7
:102F2000FFF758F906B010BD3038024000000240EB
:102F300070B504460125E07908B9002506E0E0797E
:102F4000022801D1012501E0FDF716FD2946D4F83C
:102F5000E00403F086FDD4F8E00403F02DFD70BD1D
:102F600010B50446D4F8E00403F05CFD10BD10B5C4
:102F70000446D4F8E00403F060FD10BD70B50446CB
:102F80000D4600BF94F89404012801D1022070BDC1
:102F9000012084F8940400BF65742946206804F079
:102FA000FBFF00BF002084F8940400BF00BFEEE7E1
:102FB00010B5044604F29C41D4F8E00403F068FD27
:102FC00010BD70B50446256800BF94F8940401282C
:102FD00001D1022070BD012084F8940400BFE8688C
:102FE00000F0400030B1607B012803D1A86B40F4B1
:102FF0008030A863206804F0BBFE206804F076FAF5
:1030000000BF002084F8940400BF00BFE2E7000086
:1030100010B50446D4F8E00403F097FD2068D0F81A
:10302000000E40F001002168C1F8000EE07A28B1DE
:103030000348006840F006000149086010BD000028
:1030400010ED00E070B504460D460CB9012070BDCE
:103050005848006800F00700A84209D255490D7091
:103060000846006800F00700A84201D00120EEE702
:10307000207800F0020002281DD1207800F0040022
:10308000042805D14C48006840F4E0504A490860E3
:10309000207800F00800082805D14748006840F46F
:1030A0006040454908604448006820F0F000A1688D
:1030B000084341490860207800F00100A8B3606827
:1030C000012807D13C4808380068C0F34040B8B92F
:1030D0000120BCE76068022802D06068032807D19D
:1030E000354808380068C0F3406048B90120AEE7B1
:1030F000314808380068C0F3400008B90120A6E74D
:103100002D48006820F00300616808432A490860E0
:10311000FEF7E0FF064609E0FEF7DCFF801B41F208
:103120008831884202D9032091E707E022480068ED
:1031300000F00C006168B0EB810FEDD11D48006814
:1031400000F00700A84209D91A490D700846006826
:1031500000F00700A84201D0012078E7207800F0B5
:103160000400042807D11448006820F4E050E16806
:10317000084311490860207800F00800082808D1A9
:103180000D48006820F46040216940EAC1000A4906
:10319000086000F03FF808490968C1F30311074AC5
:1031A000515CC8400649086006480068FEF7C2FF47
:1031B00000204CE7003C02400838024000B3000801
:1031C0007C00002074000020014800687047000067
:1031D0007C00002000B5FFF7F7FF04490968C1F340
:1031E0008221034A515CC84000BD000008380240FB
:1031F00010B3000800B5FFF7E7FF04490968C1F301
:103200004231034A515CC84000BD0000083802400A
:1032100010B300082DE9F047002400250026A14640
:103220002548006800F00C0020B1042805D00828CB
:103230003AD105E0DFF8849039E0DFF8849036E099
:103240001D48001F006800F03F041B48001F006875
:1032500000F4800078B11A481749091F0968C1F3C2
:103260008811A0FB01700146224600233846FDF775
:103270007BF805460EE011480F49091F0968C1F3A4
:103280008811A0FB01700146224600233846FDF755
:103290006BF805460848001F0068C0F30140401C59
:1032A0004600B5FBF6F902E0DFF8109000BF00BF62
:1032B0004846BDE8F0870000083802400024F400CA
:1032C000001BB700F8B504460CB90120F8BD207802
:1032D00000F00100002874D0F948006800F00C00EC
:1032E00004280DD0F648006800F00C00082813D11F
:1032F000F348001F006800F48000B0F5800F0BD188
:10330000EF4808380068C0F34040002859D0606892
:10331000002856D10120D9E700BF6068B0F5803F92
:1033200008D1E7480838006840F48030E44908399B
:1033300008601EE06068B0F5A02F0DD1E0480838A5
:10334000006840F48020DE490839086008460068BB
:1033500040F4803008600CE0D9480838006820F458
:103360008030D749083908600846006820F480207A
:10337000086000BF606890B1FEF7ACFE054606E04D
:10338000FEF7A8FE401B642801D903209EE7CC4825
:1033900008380068C0F340400028F1D011E0FEF783
:1033A00099FE054606E0FEF795FE401B642801D90C
:1033B00003208BE7C24808380068C0F3404000286B
:1033C000F1D1207800F0020002285FD1BC480068EB
:1033D00000F00C0058B1BA48006800F00C00082852
:1033E0001CD1B748001F006800F48000B0B9B44891
:1033F00008380068C0F3400020B1E068012801D01F
:10340000012063E7AE480838006820F0F800216921
:1034100040EAC100AA490839086037E0E06800B313
:103420000120A8490860FEF755FE054606E0FEF7B4
:1034300051FE401B022801D9032047E7A048083865
:103440000068C0F340000028F1D09D4808380068AB
:1034500020F0F800216940EAC10099490839086064
:1034600014E0002097490860FEF734FE054606E0A8
:10347000FEF730FE401B022801D9032026E79048C2
:1034800008380068C0F340000028F1D1207800F02F
:10349000080008282CD16069A8B101208A49086079
:1034A000FEF718FE054606E0FEF714FE401B022854
:1034B00001D903200AE782486C300068C0F340005D
:1034C0000028F1D014E000207F490860FEF702FEDA
:1034D000054606E0FEF7FEFD401B022801D9032049
:1034E000F4E677486C300068C0F340000028F1D162
:1034F000207800F00400042870D10027704838308C
:10350000006800F0805090B900BF002000906C4827
:103510003830006840F0805069493831086008460A
:10352000006800F08050009000BF00BF012767488E
:10353000006800F48070B0B96448006840F480709E
:1035400062490860FEF7C6FD054606E0FEF7C2FDCB
:10355000401B022801D90320B8E65C48006800F44B
:1035600080700028F2D000BFA068012808D154481C
:103570006830006840F001005149683108601DE082
:10358000A06805280DD14E486830006840F004005E
:103590004B49683108600846006840F00100086047
:1035A0000CE047486830006820F001004449683169
:1035B00008600846006820F00400086000BFA068AA
:1035C000A8B1FEF787FD054609E0FEF783FD401B25
:1035D00041F28831884202D9032077E626E0384854
:1035E00068300068C0F340000028EED013E0FEF71A
:1035F00071FD054608E0FEF76DFD401B41F2883184
:10360000884201D9032061E62D4868300068C0F384
:1036100040000028EFD1012F07D129483830006839
:1036200020F0805026493831086000BFA06900288A
:1036300045D02348006800F00C0008285DD0A06940
:10364000022845D100201F490866FEF743FD0546C4
:1036500006E0FEF73FFD401B022801D9032035E6B6
:10366000174808380068C0F340600028F1D1D4E959
:1036700007010843616A40EA81110122A06AC2EB96
:10368000500041EA00412C20005D41EA00600C49F5
:10369000091F086001200B490866FEF71BFD05465F
:1036A00006E0FEF717FD401B022801D903200DE6B6
:1036B000034808380068C0F340600028F1D049E0B2
:1036C0000838024000004742800E47420070004028
:1036D000002021490866FEF7FDFC054606E0FEF7DE
:1036E000F9FC401B022801D90320EFE51B480068C4
:1036F000C0F340600028F2D12CE0A069012800D17D
:10370000E4E51648001D0668A069012820D006F4EB
:103710008001E06981421BD106F03F01206A8142AD
:1037200016D147F6C0703040616AB0EB811F0FD1EF
:1037300006F440310122A06AC2EB5000B1EB004F09
:1037400006D106F070612C20005DB1EB006F01D056
:103750000120BBE50020B9E50000474200380240E7
:1037600070B504462546681EB0F1807F01D3012064
:103770000FE0681E4FF0E02148610F214FF0FF304D
:1037800004F008FD00204FF0E02188610720086167
:10379000002070BD10B50346002200BF93F83C0026
:1037A000012801D1022010BD012083F83C0000BF98
:1037B00022F0FF00CC6840EA040222F440708C68DA
:1037C00040EA040222F480604C6840EA040222F4D9
:1037D00000600C6840EA040222F480500C6940EA60
:1037E000040222F400504C6940EA040222F48040B2
:1037F000CC6940EA04021868426400BF002083F8E4
:103800003C0000BF00BFCEE730B502460B4600BF0C
:1038100092F83C00012801D1022030BD012082F83D
:103820003C0000BF022082F83D0010684468106828
:10383000816824F070041868044310684460184DCF
:103840001068A8421BD01068B0F1804F17D0154DFA
:103850001068A84213D0144D1068A8420FD0134D21
:103860001068A8420BD0124D1068A84207D0114D25
:103870001068A84203D0104D1068A84205D121F06D
:1038800080015868014310688160012082F83D0082
:1038900000BF002082F83C0000BF00BFBDE7000071
:1038A000000001400004004000080040000C0040FF
:1038B00000040140004001400018004010B586B0EF
:1038C0000446142101A8FCF713FE11492068884220
:1038D0001CD100BF002000900E48006840F010008E
:1038E0000C4908600846006800F01000009000BF16
:1038F00000BF481501900220029000200390049020
:103900000120059001A90448FEF7E4FA06B010BDB5
:103910000000014030380240001002402DE9F04123
:1039200004460D461646002700BF94F83C000128C7
:1039300002D10220BDE8F081012084F83C0000BFE4
:1039400036B1042E1BD0082E31D00C2E5ED145E0AE
:103950002946206801F0CAFA2068806940F0080012
:10396000216888612068806920F0040021688861EE
:1039700020688069296908432168886148E02946F0
:10398000206801F0EBFA2068806940F4006021684B
:1039900088612068806920F48060216888612068DF
:1039A0008069296940EA01202168886130E0294660
:1039B000206801F011FB2068C06940F00800216810
:1039C000C8612068C06920F004002168C8612068CF
:1039D000C069296908432168C86119E0294620683F
:1039E00001F036FB2068C06940F400602168C861BE
:1039F0002068C06920F480602168C8612068C069BF
:103A0000296940EA01202168C86101E0012700BF5F
:103A100000BF00BF002084F83C0000BF384689E7A3
:103A200010B504460CB9012010BD94F83D0028B92A
:103A3000002084F83C00204600F026F8022084F89C
:103A40003D00211D206801F0DDF9012084F84600C9
:103A500000BF84F83E0001213F2001554020015560
:103A60004120015500BF00BF012084F842004320DF
:103A70000155442001554520015500BF012084F81F
:103A80003D000020D0E7000008B50A4A01689142D5
:103A90000FD100BF002100910749096841F00101E1
:103AA000054A11601146096801F00101009100BF4B
:103AB00000BF08BD000001404438024070470000CC
:103AC00070B50546284601F07BFC0446042C0DD059
:103AD00004EBC400064901EB8000406930B104EBFF
:103AE000C401034A02EB81014869804770BD0000B0
:103AF000A86A002070B50546284601F061FC04461E
:103B0000042C0DD004EBC400064901EB8000C06911
:103B100030B104EBC401034A02EB8101C86980475C
:103B200070BD0000A86A002070B50546284601F067
:103B300047FC0446042C0DD004EBC400064901EBFD
:103B40008000806930B104EBC401034A02EB8101BB
:103B50008869804770BD0000A86A002070B50546DE
:103B6000284601F02DFC0446042C0DD004EBC400C3
:103B7000064901EB8000006930B104EBC401034A3F
:103B800002EB81010869804770BD0000A86A00202F
:103B90002DE9F84F0446206805682068C66820684B
:103BA00047694FF00009CA4605F00F09B9F1000F47
:103BB0000AD105F0200038B106F0200020B12046DF
:103BC00001F040FCBDE8F88FB9F1000F7CD007F0A0
:103BD000010018B906F49070002875D005F00100B6
:103BE00030B106F4807018B1606C40F00100606480
:103BF00005F0040030B107F0010018B1606C40F02E
:103C00000200606405F0020030B107F0010018B155
:103C1000606C40F00400606405F0080048B106F0F4
:103C2000200010B907F0010018B1606C40F00800E6
:103C30006064606C002846D005F0200028B106F0D2
:103C4000200010B1204601F0FDFB20684069C0F360
:103C5000801A606C00F0080010B9BAF1000F2DD086
:103C6000204601F053FB2068406900F040004028E6
:103C700020D100BF00BF2168143151E8001F21F09E
:103C800040002168143141E80002002AF3D100BF4E
:103C9000E06B50B17748E16B0865E06BFDF712FF10
:103CA00088B1E06B016D88470DE02046A16D884723
:103CB00009E009E02046A16D884704E02046A16D97
:103CC0008847002060647DE7206B012878D105F0EB
:103CD0001000002874D006F010000028FAD000BFB1
:103CE00000200090206800680090206840680090E4
:103CF00000BF00BF2068406900F04000402860D14C
:103D0000E06B006840681FFA80F8B8F1000F56D0E9
:103D1000A08D404553DDA4F82E80E06BC069B0F55E
:103D2000807F43D000BF00BF21680C3151E8001FE5
:103D300021F4807021680C3141E80002002AF3D19F
:103D400000BF00BF00BF2168143151E8001F21F0FF
:103D500001002168143141E80002002AF3D100BFBC
:103D600000BF00BF2168143151E8001F21F040005E
:103D70002168143141E80002002AF3D100BF20205D
:103D800084F842000020206300BF00BF21680C318E
:103D900051E8001F21F0100021680C3141E80002B9
:103DA000002AF3D100BFE06BFDF736FE022060630E
:103DB000A08DE38DC01A81B22046E26E904701E7E4
:103DC00042E0A08DE18D401A1FFA80F8E08DD0B35B
:103DD000B8F1000F37D000BF00BF21680C3151E8A7
:103DE000001F21F4907021680C3141E80002002A84
:103DF000F3D100BF00BF00BF2168143151E8001F9C
:103E000021F001002168143141E80002002AF3D1B9
:103E100000BF202084F842000020206300BF00BFC4
:103E200021680C3151E8001F21F0100021680C318D
:103E300041E80002002AF3D100BF0220606341463E
:103E40002046E26E9047BDE605F0800030B106F0F6
:103E5000800018B1204601F0EDFCB3E605F040000B
:103E600030B106F0400018B1204601F085FAA9E60D
:103E700000BFA7E6D151000810B504460CB90120D7
:103E800010BDA06900B100E000BF94F8410060B926
:103E9000002084F84000204601F0AEFA206F08B9F7
:103EA000164820672046216F8847242084F8410067
:103EB0002068C06820F400502168C860204601F0E6
:103EC0003FFB2068006920F4904021680861206869
:103ED000406920F02A00216848612068C06840F4E9
:103EE00000502168C86000206064202084F84100F0
:103EF00084F842000020606300BFC1E7013F000872
:103F000010B586B00446142101A8FCF7F1FAA849BF
:103F10002068884274D100BF00200090A548006846
:103F200040F01000A34908600846006800F0100047
:103F3000009000BF00BF00BF002000909D481438D3
:103F4000006840F002009B49143908600846006888
:103F500000F00200009000BF00BF00BF00200090F2
:103F60000846006840F0010008600846006800F05C
:103F70000100009000BF00BF80200190022002904D
:103F800000200390032004900720059001A98A488F
:103F9000FDF7A0FF4FF40070019002200290002076
:103FA0000390032004900720059001A98348FDF7A2
:103FB00091FF8348834908604FF00060486000210A
:103FC00080488160C1604FF48061016100214161DE
:103FD0008161C16101624162FDF7A8FE08B1FCF791
:103FE000CBFC00BF7748E063846300BF002205215B
:103FF0002520FEF703F92520FEF7ECF8D6E0FFE7D1
:1040000071492068884258D100BF0020009069485B
:10401000001F006840F480206649091F08600846B8
:10402000006800F48020009000BF00BF00BF0020A7
:10403000009060481438006840F004005D4914396D
:1040400008600846006800F00400009000BF00BF50
:104050004FF4406001900220029000200390032062
:1040600004900720059001A95848FDF733FF5848F0
:10407000584908604FF00060486000215548816051
:10408000C1604FF480610161002141618161C161C2
:1040900001624162FDF74AFE08B1FCF76DFC00BF0A
:1040A0004C48E063846300BF002205212720FEF70F
:1040B000A5F82720FEF78EF878E047492068884267
:1040C00074D100BF002000903A48006840F0200002
:1040D000384908600846006800F02000009000BFE2
:1040E00000BF00BF0020009032481438006840F044
:1040F00040003049143908600846006800F040006C
:10410000009000BF00BF4FF4844001900220029055
:1041100000200390032004900820059001A92F4857
:10412000FDF7D8FE264818382D49086080054860FC
:1041300000212B488160C1604FF480610161002142
:1041400041618161C16101624162FDF7EFFD08B12A
:10415000FCF712FC00BF2248E063846300BF1848EC
:104160006030204908604FF02060486040211D48C1
:1041700081600021C1604FF48061016100214161D3
:104180008161C16101624162FDF7D0FD08B1FCF7B8
:10419000F3FB00BF1348A063846300BF0022052126
:1041A0004720FEF72BF84720FEF714F806B010BDA5
:1041B0000010014044380240000402400000024068
:1041C000406402400C040020004800400008024007
:1041D000286002406C0400200014014000180240D6
:1041E000CC0400202C05002070B504460D46164670
:1041F00094F8420020280BD105B10EB9012070BD02
:104200000020206332462946204601F0AFFAF6E747
:104210000220F4E710B5034600242AB9586C40F098
:1042200020005864012010BD93F84100202825D1BA
:104230000D291CD2DFE801F007090B0D0F11131532
:104240001B1B1B1719009A6417E0DA6415E01A6546
:1042500013E05A6511E09A650FE0DA650DE01A6621
:104260000BE05A6609E01A6707E05A6705E0586CE8
:1042700040F020005864012400BF17E093F841008B
:1042800078B90B2902D00C2904D101E01A6707E0A4
:104290005A6705E0586C40F020005864012400BFC4
:1042A00004E0586C40F02000586401242046BAE72E
:1042B00070B505460E21154804F050F90446134820
:1042C000807BE1B2884204D11048C07BB0EB142F50
:1042D0000BD00122D1020E48FDF7F6FE00224FF46A
:1042E00080510B48FDF7F0FE70BD0122D102084855
:1042F000FDF7EAFE00224FF480510548FDF7E4FE89
:104300000248FCF7ADFB00BFEEE70000D86C0020D0
:10431000001C024070B50546284601F051F80446DD
:10432000042C0DD004EBC400064901EB800080682A
:1043300030B104EBC401034A02EB81018868804775
:1043400070BD0000A86A002010B5034693F8410034
:10435000202813D101B10AB9012010BD19629A8435
:10436000DA8400205864212083F841001868C0686E
:1043700040F080001C68E0600020EEE70220ECE7DF
:1043800070B50546284601F01BF80446042C0DD0F4
:1043900004EBC400064901EB8000406830B104EB37
:1043A000C401034A02EB81014868804770BD0000E8
:1043B000A86A002070B50546284601F001F80446B9
:1043C000042C0BD004EBC400054951F8200028B19F
:1043D00004EBC401024A52F82100804770BD00007E
:1043E000A86A002000BFFEE730B50B46002100BFE1
:1043F00016E00A24B4EB107F05D9302404EB1074C6
:1044000003F8114005E0412404EB10740A3C03F862
:104410001140000100254C00641C1D554C1CE1B2EC
:104420009142E6DB30BD000010B50E480E49086031
:104430000320486000210C488160C1604FF41021C6
:1044400001614FF4001141610021017641768176CE
:10445000C17601774177FCF7DEFF08B1FCF78CFAF3
:1044600010BD0000006400400C02002010B50E4892
:104470000E4908600320486000210C488160C1603B
:104480004FF4102101614FF40011416100210176C8
:1044900041768176C17601774177FCF7BCFF08B1A0
:1044A000FCF76AFA10BD00000068004034020020EA
:1044B00008B500BF002000901E48006840F40010BE
:1044C0001C4908600846006800F40010009000BF16
:1044D00000BF00BF002000900846006840F4800044
:1044E00008600846006800F48000009000BF00BF2C
:1044F000002205210C20FDF781FE0C20FDF76AFE4D
:10450000002205213920FDF779FE3920FDF762FEF2
:10451000002205213A20FDF771FE3A20FDF75AFEF0
:10452000002205214520FDF769FE4520FDF752FEDA
:1045300008BD00003038024010B5074A0021074886
:1045400004F036FB06490860064A0021064804F0DC
:104550002FFB0649086010BDD4B200081B4D0008AF
:104560000400002018B70008D950000800000020FF
:1045700000B587B0142102A8FBF7BAFF00BF0020E6
:1045800001903D48006840F002003B490860084641
:10459000006800F00200019000BF00BF00BF0020D3
:1045A00001900846006840F0400008600846006836
:1045B00000F04000019000BF00BF00BF002001904C
:1045C0000846006840F0010008600846006800F0F6
:1045D0000100019000BF00BF00BF0020019008460D
:1045E000006840F0080008600846006800F0080015
:1045F000019000BF00BF00BF002001900846006886
:1046000040F0040008600846006800F004000190D3
:1046100000BF00BF00BF002001900846006840F0C6
:10462000800008600846006800F08000019000BF2C
:1046300000BF00BF002001900846006840F0100055
:1046400008600846006800F01000019000BF00BF3D
:1046500000224FF4E0510948FDF736FD4FF4E050D9
:1046600002900120039000200490059002A90348C5
:10467000FDF730FC07B000BD30380240001C02409E
:1046800000B591B000200F9010901C2108A8FBF7F6
:104690002FFF20216846FBF72BFF234823490860A2
:1046A000A720486000212148816044F61F61C16055
:1046B0000021016141618161FFF7B2F908B1FCF7A6
:1046C0005BF900200F9010900FA91848FFF79CF895
:1046D00008B1FCF751F960200890002009900A9079
:1046E0000B900C900D900E90002208A90F48FFF738
:1046F00015F908B1FCF740F90020009001900290F4
:10470000039004904FF400500590002007906946F4
:104710000648FFF73FF808B1FCF72EF90348FFF70A
:10472000CDF811B000BD0000000001405C02002087
:1047300010B50A480A4908600A484860002108483C
:104740008160C16001610C21416100218161C16111
:10475000FFF792FB08B1FCF70FF910BD0010014004
:10476000A402002000093D0010B50C480C49086067
:104770000C48486000210A4881604FF40051C16034
:10478000002101610C21416100218161C161FFF7BC
:1047900073FB08B1FCF7F0F810BD000000480040C2
:1047A0001C030020A086010010B50A480A490860D1
:1047B0000A484860002108488160C16001610C21FD
:1047C000416100218161C161FFF756FB08B1FCF72F
:1047D000D3F810BD001401409403002000093D00EF
:1047E00010B500220D490E4801F0B7FE08B1FCF7E4
:1047F000C3F80C490A4802F0E9F908B1FCF7BCF823
:104800000949074801F0E0FA08B1FCF7B5F8044897
:1048100002F0DEFA08B1FCF7AFF810BD0C00002082
:104820008C050020100100205C00002000BFFEE786
:1048300000BFFEE710B50248FDF7FFFE10BD000007
:10484000681A002010B5034A08210120FBF708FF71
:10485000002010BD058100082DE9F04704460D46F3
:1048600026683746D6F8408007F5306000EB4510E3
:10487000D0F80890104880450BD909F40040B0F5F5
:10488000004F06D14FF4004107F5306000EB4510B2
:1048900081602046FEF78CFB0748804508D9A07947
:1048A000012805D104F29C420121206802F03EFF5C
:1048B0000020BDE8F08700000A30544F2DE9F04792
:1048C00005460C46D5F800904E46D9F840A006F5AE
:1048D000306000EB4410D0F80880A879012855D149
:1048E00008F0080008280FD1434882450BD908F486
:1048F0000040B0F5004F7BD14FF4004106F5306029
:1049000000EB4410816073E008F02000202806D1FD
:10491000202106F5306000EB4410816068E008F06B
:104920002800002864D1344882450CD908F400409E
:10493000B0F5004F07D14FF4004106F5306000EBB1
:104940004410816054E004EBC40105F5157000EBE0
:10495000810706F5306000EB4410396A0069C0F346
:104960001200081A786164B9386930B905F29C42BE
:104970000121286802F0DAFE03E07969F86808444A
:10498000F860E1B22846FDF7CFFC31E01B488245D4
:104990001BD108F40040B0F5004F07D14FF400419F
:1049A00006F5306000EB4410816021E008F0200043
:1049B000202805D1202106F5306000EB44108160ED
:1049C000E1B22846FDF7B0FC12E06CB904EBC4017B
:1049D00005F5157000EB8100006928B905F29C42CD
:1049E0000021286802F0A2FEE1B22846FDF79CFCF7
:1049F0000020BDE8F08700000A30544F0A31544FC0
:104A00002DE9F84F07460E46D7F80090C84606EB4A
:104A1000C60107F1140000EB8104D4E904108842B8
:104A200002D90120BDE8F88FD4E90401451AA06835
:104A3000A84200D2A568E81C4FEA900A17E0D4E922
:104A40000401451AA068A84200D2A568E81C4FEAF4
:104A5000900AB879ABB2F2B200904846E16803F030
:104A60002DFBE0682844E06060692844606108F537
:104A7000106000EB4610806980B2504506D3D4E93F
:104A80000410884202D220690028D8D1D4E9040158
:104A900088420ED806F00F01012000FA01FB40F613
:104AA000340050F8080020EA0B0040F6340141F8C9
:104AB00008000020B6E70000B0EE401A10B99FEDE4
:104AC000790A704790ED100A80ED110A90ED0F0AF7
:104AD00080ED100AC0ED060A80ED071A30EEC10A1B
:104AE00080ED0F0A0178002975D190ED010AD0ED13
:104AF0000F1A20EE210A80ED090A90ED0A0AD0ED86
:104B0000021A90ED0F2A01EE820A80ED0A0A90ED5A
:104B10000D0A80ED0E0A90ED0C0A80ED0D0A90ED65
:104B20000F0AD0ED101A30EE610A80ED0C0A90EDFC
:104B3000030AD0ED0C1A20EE210A80ED0B0A90ED4D
:104B40000A0AD0ED051AB4EEE10AF1EE10FA04DD1E
:104B500090ED050A80ED0A0A10E090ED0A0AD0ED0A
:104B6000051AF1EE611AB4EEE10AF1EE10FA05D27F
:104B700090ED050AB1EE400A80ED0A0A90ED090AAF
:104B8000D0ED0A1A30EE210AD0ED0B1A30EE210AD0
:104B900080ED080A90ED080AD0ED041AB4EEE10A9F
:104BA000F1EE10FA04DD90ED040A80ED080A76E0DB
:104BB00090ED080AD0ED041AF1EE611AB4EEE10AA4
:104BC000F1EE10FA6BD290ED040AB1EE400A80EDDE
:104BD000080A64E0FFE70178012960D190ED0F0A2F
:104BE000D0ED101A30EE610AD0ED011A20EE210A44
:104BF00080ED090A90ED020AD0ED0F1A20EE210A8D
:104C000080ED0A0A90ED0D0A80ED0E0A90ED0C0A77
:104C100080ED0D0A90ED0F0AD0ED101AB0EE002ACB
:104C200002EE610AD0ED111A30EE210A80ED0C0A75
:104C300090ED030AD0ED0C1A20EE210A80ED0B0A4C
:104C400090ED090AD0ED0A1A30EE210AD0ED0B1AC8
:104C500030EE210AD0ED081A30EE210A80ED080A64
:104C600090ED080AD0ED041AB4EEE10AF1EE10FA64
:104C700004DD90ED040A80ED080A10E090ED080ACA
:104C8000D0ED041AF1EE611AB4EEE10AF1EE10FA79
:104C900005D290ED040AB1EE400A80ED080A90EDCD
:104CA000080A0EE70000000000B102B97047017069
:104CB00092ED001A80ED011A92ED011A80ED021AB0
:104CC00092ED021A80ED031A80ED040AC0ED050A88
:104CD0009FED0C1A80ED0E1A80ED0D1A80ED0C1A66
:104CE0009FED081A80ED081A80ED0B1A80ED0A1A64
:104CF00080ED091A80ED111A80ED101A80ED0F1A5F
:104D000000BFD3E70000000030B501460A46137823
:104D1000521C147843EA042030BD10B5FFF760FD43
:104D200000BF012003F034FEFBE710B5FDF7D8F912
:104D300005F016FF012801D005F04CFB10BD000066
:104D400000B593B0302107A8FBF7D2FB142102A8CD
:104D5000FBF7CEFB00BF002001902348006840F025
:104D60008050214908600846006800F0805001909A
:104D700000BF00BF00BF002001901C48006840F445
:104D800080401A4908600846006800F4804001909D
:104D900000BF00BF012007900004089002200D9082
:104DA00041050E9106210F91482110910221119188
:104DB0000421129107A8FEF785FA08B1FBF7DCFD84
:104DC0000F20029002200390002004904FF48050A6
:104DD000059000200690022102A8FEF733F908B1E1
:104DE000FBF7CAFD13B000BD403802400070004020
:104DF0000348006840F470000149086070470000F3
:104E000088ED00E010B502682D4B98420ED0B0F14D
:104E1000804F0BD02B4B984208D02B4B984205D09B
:104E20002A4B984202D02A4B984203D122F07002BA
:104E30004B681A43224B984220D0B0F1804F1DD0CE
:104E4000204B98421AD0204B984217D01F4B9842C3
:104E500014D01F4B984211D01E4B98420ED01E4BBF
:104E600098420BD01D4B984208D01D4B984205D05C
:104E70001C4B984202D01C4B984203D122F4407242
:104E8000CB681A4322F080034C6943EA04020260B3
:104E90008B68C3620B688362094B984202D00C4B4B
:104EA000984201D10B69036301234361036903F055
:104EB00001031BB1036923F00103036110BD00006E
:104EC000000001400004004000080040000C0040C9
:104ED00000040140004001400044014000480140FE
:104EE00000180040001C00400020004030B5026A5D
:104EF000056A25F0010505624368846924F07004A1
:104F000024F003040D682C4322F002028D682A432A
:104F1000104DA84200D103E00F4DA84206D100BFBA
:104F200022F00802CD682A4322F00402094DA8426B
:104F300002D0094DA84207D123F4807323F40073F3
:104F40004D692B438D692B43436084614D684563F4
:104F5000026230BD000001400004014030B5026A29
:104F6000056A25F0100505624368846924F4E0446D
:104F700024F440740D6844EA052422F020028D6870
:104F800042EA0512124DA84200D103E0114DA84299
:104F900007D100BF22F08002CD6842EA051222F05C
:104FA00040020B4DA84202D00A4DA84209D123F479
:104FB000806323F400634D6943EA85038D6943EA06
:104FC0008503436084614D688563026230BD0000E3
:104FD000000001400004014030B5026A056A25F472
:104FE000807505624368C46924F0700424F00304EA
:104FF0000D682C4322F400728D6842EA0522124D9E
:10500000A84200D103E0114DA84207D100BF22F40D
:105010000062CD6842EA052222F480620A4DA8426D
:1050200002D00A4DA84209D123F4805323F400533F
:105030004D6943EA05138D6943EA05134360C46172
:105040004D68C563026230BD0000014000040140AC
:1050500030B5036A056A25F4805505624468C26963
:1050600022F4E04222F440720D6842EA052223F461
:1050700000538D6843EA0533084DA84202D0084D1D
:10508000A84204D124F480444D6944EA8514446064
:10509000C2614D680564036230BD0000000001403C
:1050A0000004014003F0BCF8FFF7CCFB03E004F080
:1050B000ABFF03F0C1F8FAE703F0F8FA012211039D
:1050C0000448FDF701F804E003F0BAFA012003F008
:1050D0005FFCF9E7001C024070B5054603F0F4FCE4
:1050E000154A0021154803F063FD1549C860154AAB
:1050F0000021154803F05CFD11494860134A002166
:10510000134803F055FD0E49C861124A00211248A8
:1051100003F04EFD0A490862104A0021104803F0CE
:1051200047FD0749486203F01BFD03F03BFD0446C1
:1051300003F09AFD70BD00003CB7000865510008FF
:10514000C46D002060B70008A550000884B70008AF
:1051500071510008A8B70008B1510008CCB7000889
:10516000B950000800BF4FF4FA7003F011FCFAE7E1
:1051700008B503F019FB13E00A4890ED000AB8EEF9
:10518000C00A03F03DFB084800231A461946009068
:105190000648B0F90000FBF7BFFA022003F0F8FB65
:1051A000EAE70000040200200C020020FC010020BD
:1051B0000BE004F05DFB102003F084FBFBF7B2FD75
:1051C00002490860022003F0E3FBF2E70802002036
:1051D00070B50546AC6B0020E085E0842046A16DEB
:1051E000884770BD70B505460026AC6B20684069E5
:1051F000C0F3C01694F84100212805D126B1002043
:10520000E084204600F0C8F820684069C0F38016AA
:1052100094F84200222805D126B10020E0852046DE
:1052200000F074F8606C40F0100060642046A16DDE
:10523000884770BD70B50546AC6B2868006800F4FF
:105240008070002842D1E08500BF00BF21680C318A
:1052500051E8001F21F4807021680C3141E8000200
:10526000002AF3D100BF00BF00BF2168143151E80C
:10527000001F21F001002168143141E80002002ADA
:10528000F3D100BF00BF00BF2168143151E8001FF7
:1052900021F040002168143141E80002002AF3D1D6
:1052A00000BF202084F84200206B01280ED100BFEF
:1052B00000BF21680C3151E8001F21F01000216867
:1052C0000C3141E80002002AF3D100BF00206063E6
:1052D000206B012804D1A18D2046E26E904702E0A8
:1052E0002046616D884770BD70B50546AC6B0120E6
:1052F0006063206B012805D1A08D41082046E26E35
:10530000904702E02046216D884770BD00BF00BF76
:1053100002680C3252E8002F22F4907102680C32BD
:1053200042E80013002BF3D100BF00BF00BF0268AA
:10533000143252E8002F22F001010268143242E8D0
:105340000013002BF3D100BF016B01290ED100BF68
:1053500000BF02680C3252E8002F22F010010268F0
:105360000C3242E80013002BF3D100BF202180F85B
:10537000421000210163704710B504462068C068E0
:1053800020F040002168C860202084F841002046B9
:10539000E16C8847002010BD00BF00BF02680C32DE
:1053A00052E8002F22F0C00102680C3242E80013DC
:1053B000002BF3D100BF202180F84110704700007E
:1053C00001460A4A0868904201D100207047084A05
:1053D0000868904201D10120F8E7064A0868904227
:1053E00001D10220F2E70420F0E70000004800406D
:1053F0000010014000140140094981640949C16459
:105400000949016509494165094981650949C1653C
:1054100009490166094941660949C16670470000AA
:10542000B54300088143000815430008B142000855
:105430005D3B0008C13A0008293B0008F53A000826
:10544000BD3A0008F8B5044694F84200222875D108
:10545000A068B0F5805F0CD1206950B90025A66A1C
:1054600020684068C0F308003080A06A801CA062F9
:1054700015E0A56A0026A068B0F5805F03D0A0689B
:1054800028B9206918B920684068287004E02068AD
:10549000406800F07F002870A06A401CA062E08D88
:1054A000401E80B2E085002846D12068C06820F008
:1054B00020002168C8602068C06820F480702168DE
:1054C000C8602068406920F0010021684861202000
:1054D00084F8420000206063206B012826D1002060
:1054E000206300BF00BF21680C3151E8001F21F08C
:1054F000100021680C3141E80002002AF3D100BFFE
:105500002068006800F0100010280AD100BF0020B9
:10551000009020680068009020684068009000BFFC
:1055200000BFA18D2046E26E904702E02046616DEB
:1055300088470020F8BD01E00020FBE70220F9E7E2
:105540002DE9F84F04462068006920F44050E168D6
:105550000843216808612169A0680843616908431C
:10556000E169084300902068C06849F20C618843F3
:10557000009908432168C8602068406920F44070A1
:10558000A16908432168486176492068884203D0B0
:1055900075492068884203D1FDF72CFE814602E060
:1055A000FDF718FE8146E069B0F5004F6CD102208E
:1055B0006168A0FB015003461920A9FB0070014659
:1055C0002A463846FAF7D0FE6421B0FBF1F04FEAE4
:1055D000001A02206168A0FB01510B461920A9FBAB
:1055E00000712A463846FAF7BFFE834602206168FA
:1055F000A0FB015003461920A9FB00712A4638463A
:10560000FAF7B2FE6421B0FBF1F000EBC00101EB50
:105610000010ABEB8000322101EBC0006421B0FB35
:10562000F1F000F0F8000AEB400A02206168A0FBEC
:10563000015003461920A9FB007001462A4638464E
:10564000FAF792FE834602206168A0FB01500346F0
:105650001920A9FB00712A463846FAF785FE642115
:10566000B0FBF1F000EBC00101EB0010ABEB8000F0
:10567000322101EBC0006421B0FBF1F000F0070023
:105680005044216888606AE004206168A0FB0150F2
:1056900003461920A9FB007001462A463846FAF74E
:1056A00063FE824604206168A0FB01500346192076
:1056B000A9FB007001462A463846FAF755FE6421D8
:1056C000B0FBF1F000EBC00101EB0010AAEB800091
:1056D000322101EB00106421B0FBF1F000F0F00A80
:1056E00004206168A0FB017003461920A9FB00514A
:1056F0003A462846FAF738FE6421B0FBF1F00AEB8F
:10570000001A04206168A0FB01510B461920A9FB77
:1057100000712A463846FAF727FE8346042061685E
:10572000A0FB015003461920A9FB007001462A4640
:105730003846FAF719FE6421B0FBF1F000EBC00126
:1057400001EB0010ABEB8000322101EB0010642173
:10575000B0FBF1F000F00F00504421688860BDE814
:10576000F88F0000001001400014014077B581B0AF
:10577000044615460298A062A58500206064222098
:1057800084F842002848E16BC8632848E16B08644C
:105790002748E16BC8640020E16B086502AE3268FF
:1057A0002368191D2B46E06BFCF736FB00BF002079
:1057B000009020680068009020684068009000BF5A
:1057C00000BF206970B100BF00BF21680C3151E8F3
:1057D000001F41F4807021680C3141E80002002A6A
:1057E000F3D100BF00BF00BF2168143151E8001F92
:1057F00041F001002168143141E80002002AF3D190
:1058000000BF00BF00BF2168143151E8001F41F004
:1058100040002168143141E80002002AF3D100BFA2
:10582000002004B070BD000035520008E9520008A5
:10583000E5510008014691F84100212828D18868E7
:10584000B0F5805F0BD1086948B90A6A1088C0F3C7
:1058500008000B685860086A801C086205E00B6A43
:10586000581C086218780B685860C88C401E80B2BB
:10587000C88458B90868C06820F080000B68D860F8
:105880000868C06840F040000B68D860002070478E
:105890000220FCE710B50248FEF77AF910BD0000BF
:1058A000A402002010B50348FAF7EEFE0148FEF707
:1058B0006FF910BD1C03002010B50248FEF768F90F
:1058C00010BD0000940300202DE9F04104460D4670
:1058D000D4F8C87204F53070D4F8D41250F821000E
:1058E00010B90320BDE8F08104F53070D4F8D4126B
:1058F00050F8216005F00F0000EB800104F1140066
:1059000000EB8100406838B305F00F0000EB800128
:1059100004F1140000EB8100416805F00F0000EB7A
:10592000C00207F1140000EB82008068B1FBF0F2C6
:1059300000FB121080B9002105F00F0000EB80027F
:1059400004F1140000EB8200416000231A4629464E
:10595000204601F008F917E00020C6F8140204F50B
:105960003170D4F8D41250F82100006960B1D6F833
:10597000080204F53171D4F8D42251F822102A46D5
:105980000B6906F5047198470020ABE770B5044633
:105990000E4604F53070D4F8D41250F82150D4F8E3
:1059A000D41250F8210008B9032070BD31462046BA
:1059B00000F031FFC5F80C02D5F8040204F531718E
:1059C000D4F8D43251F82310CA6805F50371904712
:1059D0000020EAE770B504460D46304801782046BD
:1059E00000F0EBFD00212D48007800F00F0000EBE7
:1059F000800204F1140000EB820001822848017843
:105A0000204600F0DAFD00212548007800F00F0064
:105A100000EB800204F5AA7000EB820001822148AD
:105A20000178204600F0C9FD00211E48007800F0F2
:105A30000F0000EB800204F1140000EB82000182F1
:105A40001848007800F00F0000EB800204F1140009
:105A500000EB8200418204F53070D4F8D41250F883
:105A60002100C8B104F53171D4F8D42251F82210C4
:105A70004868804704F53071D4F8D42251F82200E8
:105A800001F09AFB002104F53070D4F8D42240F8DC
:105A900022100020C4F8BC02002070BD8B01002041
:105AA0008C0100208D01002070B5044604F5307093
:105AB000D4F8D41250F821500DB9032070BD04F56C
:105AC0003170D4F8D41250F8210098B195F8000242
:105AD000FF280FD095F8012295F8000204F53171E6
:105AE000D4F8D46251F826108B6829469847FF20D5
:105AF00085F800020020E1E701460A2008800148FD
:105B000070470000040100202DE9F0410446822185
:105B10000D4800F06EFC054601210B4800F069FCC1
:105B200006468121084800F064FC07460DB11020AC
:105B3000A8710EB14020B0800FB14020B880432042
:105B400020800148BDE8F081480100202DE9F041A6
:105B5000044682210E4800F04CFC054601210C4809
:105B600000F047FC06468121094800F042FC074648
:105B70000DB11020A87116B14FF40070B08017B1AC
:105B80004FF40070B880432020800148BDE8F081C8
:105B9000480100202DE9F041044682210D4800F023
:105BA00028FC054601210B4800F023FC0646812114
:105BB000084800F01EFC07460DB11020A8710EB178
:105BC0004020B0800FB14020B880432020800148A1
:105BD000BDE8F0814801002070B504460E464FF440
:105BE000077001F0EBFA054645B9002104F5307065
:105BF000D4F8D42240F82210022070BD4FF407716F
:105C00002846FAF775FC04F53070D4F8D41240F841
:105C10002150D4F8D41250F82100C4F8BC02207CE2
:105C200098BB4FF40073022250480178204600F0E0
:105C300093FE01214D48007800F00F0000EB800238
:105C400004F1140000EB820001824B02022248485A
:105C50000178204600F080FE01214548007800F0E0
:105C60000F0000EB800204F5AA7000EB82000182B5
:105C700010214048007800F00F0000EB800204F192
:105C8000140000EB8200418232E0FFE74023022251
:105C900036480178204600F05FFE01213348007845
:105CA00000F00F0000EB800204F1140000EB820012
:105CB0000182402302222E480178204600F04CFE4B
:105CC00001212B48007800F00F0000EB800204F562
:105CD000AA7000EB8200018210212648007800F0B3
:105CE0000F0000EB800204F1140000EB82004182FF
:105CF000082303221F480178204600F02DFE0121D1
:105D00001C48007800F00F0000EB800204F1140042
:105D100000EB820001820020C5F8040204F5317115
:105D2000D4F8D42251F82210086880470020C5F822
:105D30001402C5F81802D5F8040208B902205CE77D
:105D4000207C48B94FF40073094801782046D5F803
:105D5000042200F019FE07E04023054801782046A0
:105D6000D5F8042200F010FE002046E78B01002049
:105D70008C0100208D01002070B5044604F53070C0
:105D8000D4F8D41250F82150D4F8D41250F821008D
:105D900008B9032070BD207C48B94FF4007309484E
:105DA00001782046D5F8042200F0EEFD07E04023FC
:105DB000044801782046D5F8042200F0E5FD0020D3
:105DC000E8E700008C010020024609B90320704773
:105DD00002F53170D2F8D43240F823100020F6E7F3
:105DE00010B5024602F53070D2F8D44250F8243093
:105DF0000BB9032010BDC3F804120020FAE730B538
:105E000003460C4603F53070D3F8D45250F82510F1
:105E100009B9032030BDC1F80842C1F810220020A2
:105E2000F8E72DE9FC4105460C4605F53070D5F83C
:105E3000D41250F82160002001900090804616B9DD
:105E40000320BDE8FC81207800F0600000283DD0F0
:105E500020287CD1E08868B3207800F08000B8B1B9
:105E6000E288607805F53171D5F8D4C251F82C106C
:105E70008B6831469847E088072801D9072000E061
:105E8000E08807463A463146284600F0E2F81CE032
:105E9000607886F80002E088402801D2E08800E0BF
:105EA000402086F8010296F801223146284600F08B
:105EB000AFF80AE0607805F53171D5F8D42251F8D1
:105EC000221000228B682146984747E0607830B165
:105ED000012832D00A2813D00B282FD121E095F8C1
:105EE0009C02032805D102226946284600F0B1F839
:105EF00005E02146284600F07FF84FF0030824E033
:105F000095F89C02032805D1012201A9284600F03A
:105F1000A0F805E02146284600F06EF84FF003088F
:105F200013E095F89C02032805D02146284600F08E
:105F300063F84FF0030808E009E006E02146284630
:105F400000F05AF84FF0030800BF00BF06E02146FA
:105F5000284600F051F84FF0030800BF00BF40464C
:105F60006FE770B504460D460026D4F8B8022946FE
:105F700042682046904700B10326304670BD70B598
:105F800004460D4694F89C02012804D0022803D050
:105F900003280CD101E000BF00BF6888012805D1AB
:105FA0000020C4F8A402204600F064F804E029466A
:105FB000204600F021F800BF00BF70BD024600205F
:105FC000704702460020704770B506460C461546DD
:105FD0002B4622460021304600F0D6FC002070BD42
:105FE00070B506460C4615462B4622460021304623
:105FF00000F0B9FD002070BD70B504460D4680214B
:10600000204600F080FD0021204600F07CFD70BDA0
:1060100070B504460E4615460320C4F894024FF4AA
:10602000AC700551001D05512B463246002120461B
:1060300000F0AAFC002070BD10B504460520C4F88D
:10604000940200231A461946204600F09DFC0020C9
:1060500010BD70B504460E4615460220C4F89402E1
:10606000A561E5612B4632460021204600F07BFD0C
:10607000002070BD10B504460420C4F8940200232B
:106080001A461946204600F06EFD002010BD0000A3
:1060900070B505460C462DB92246064906A000F00B
:1060A00012FA04E02246034903A000F00CFA01486A
:1060B00070BD00006808002043444320436F6E66B3
:1060C00069670000024612200880014870470000FE
:1060D0002800002070B505460C462DB92246064919
:1060E00006A000F0F0F904E02246034903A000F006
:1060F000EAF9014870BD00006808002043444320CD
:10610000496E746572666163650000000246042092
:1061100008800148704700003C00002070B505462B
:106120000C462246024903A000F0CDF9004870BD9C
:106130006808002053544D6963726F656C65637421
:10614000726F6E696373000070B505460C462DB919
:106150002246064906A000F0B6F904E022460349AB
:1061600003A000F0B0F9014870BD000068080020ED
:1061700053544D3332205669727475616C20436FED
:106180006D506F727400000070B505460C461A2001
:106190002080FAF7CBFD014870BD000040000020D0
:1061A00070B504460D46E888012804D029462046EB
:1061B000FFF722FF1EE094F89C02012804D0022879
:1061C00003D0032810D109E000BF0020A060012205
:1061D00004F108012046FFF73CFF0AE00122211DDF
:1061E0002046FFF736FF04E029462046FFF704FF6C
:1061F00000BF00BF70BDF8B504460E4600200090F9
:106200000027002570880012082875D2DFE800F00A
:10621000C7040C20C7C7A5B5207CD4F8B4120A68FF
:10622000694690470746C1E0207C40B9D4F8B802DF
:10623000816A6846884707460220787007E0D4F8EC
:10624000B802C16A68468847074602207870ADE008
:10625000B078062878D2DFE800F00316293C5063B6
:10626000D4F8B402406838B1207CD4F8B4124A683B
:1062700069469047074605E031462046FFF7BCFED9
:10628000681CC5B267E0D4F8B402806838B1207CDD
:10629000D4F8B4128A6869469047074605E031464B
:1062A0002046FFF7A9FE681CC5B254E0D4F8B4023A
:1062B000C06838B1207CD4F8B412CA6869469047E7
:1062C000074605E031462046FFF796FE681CC5B23A
:1062D00041E0D4F8B402006938B1207CD4F8B4129B
:1062E0000A6969469047074605E031462046FFF7B0
:1062F00083FE681CC5B22EE051E0D4F8B4024069B8
:1063000038B1207CD4F8B4124A69694690470746F0
:1063100005E031462046FFF76FFE681CC5B21AE063
:10632000D4F8B402806940B1207CD4F8B4128A69F0
:1063300069469047074606E006E031462046FFF7EB
:106340005BFE681CC5B206E031462046FFF754FEEE
:10635000681CC5B200BF00BF28E0207C30B9D4F86B
:10636000B802416B68468847074605E0314620463B
:10637000FFF742FE681CC5B218E0207C40B9D4F893
:10638000B802016B6846884707460720787005E029
:1063900031462046FFF730FE681CC5B206E03146A4
:1063A0002046FFF729FE681CC5B200BF00BF05B13B
:1063B000F8BDF088C0B1BDF8000080B1F088BDF82C
:1063C0000010884202DDBDF8000000E0F088009077
:1063D000BDF8002039462046FFF73BFE07E0314676
:1063E0002046FFF709FE02E02046FFF743FE00BF0C
:1063F000DEE72DE9F84105460F462C462E464FF0C4
:10640000000870883178884218DD307800900FE0FD
:106410006946204600F020F804466078052807D138
:10642000A04698F80200B84200D106E04FF00008FC
:106430007088BDF800108842EADC00BF4046BDE825
:10644000F881014600200A4602E0431CD8B2521CE3
:106450001378002BF9D1704710B5024610460B880F
:10646000047823440B800378981810BD70B5044657
:106470000D4694F89C02012804D0022803D003287A
:106480001AD101E000BF00BFE888022804D02946E5
:106490002046FFF7B1FD14E00120E060D4F8A4022B
:1064A00018B1E06840F00200E060022204F10C0143
:1064B0002046FFF7CEFD04E029462046FFF79CFD6D
:1064C00000BF00BF70BD2DE9F04107460D46904664
:1064D00000240FB9BDE8F0813E463046FFF7B1FF1A
:1064E000022101EB4000B0F5007F01D9080204E071
:1064F0003046FFF7A6FF4000801CA8F8000098F87F
:1065000000002855601CC4B203202855601CC4B28A
:1065100008E030782855761C601CC4B2002028554D
:10652000601CC4B230780028F3D100BFD2E7014626
:10653000002031B1012906D0022906D0032908D153
:1065400005E0002007E0032005E0012003E0032030
:1065500001E0032000BF00BF70472DE9F041044671
:106560000D46164614B90320BDE8F0810020C4F89A
:10657000B802C4F8C402C4F8D0020DB1C4F8B452D1
:10658000012084F89C022670204600F04DF9074651
:106590003846E9E72DE9F04104460D46002600277C
:1065A0002946D4F8C802FBF72CFF06463046FFF711
:1065B000BEFF07463846BDE8F0812DE9F0410446AC
:1065C0000D46002600272946D4F8C802FBF7E4FE52
:1065D00006463046FFF7ABFF07463846BDE8F08178
:1065E0002DE9F04704460F469146002F56D104F19D
:1065F0001405D4F89402022846D1D5E90201884254
:106600000FD9D5E90201401AA86049462046AA6878
:10661000FFF7E6FC00231A461946204600F0B4F9BD
:1066200032E0D5E90210884217D1E96868688842EB
:1066300013D36868D4F8981288420ED2002211460B
:106640002046FFF7CDFC0020C4F8980200231A462C
:106650001946204600F098F916E094F89C020328A9
:106660000BD1D4F8B802C06838B10020C4F8D40205
:10667000D4F8B802C168204688478021204600F03F
:1066800042FA2046FFF7D8FC94F8A00250B3204607
:1066900000F0C0FA002084F8A00223E047F0800157
:1066A0002046FFF78BFC0646FF2E1BD0D6B994F888
:1066B0009C02032816D104F52E7050F8260040697C
:1066C00080B1C4F8D46204F52E7050F82600394623
:1066D0004269204690478046B8F1000F02D04046FC
:1066E000BDE8F0870020FBE72DE9F04705460F469F
:1066F00090464FF00009002F51D105F5AA76D5F844
:10670000940203286FD1D6E90201884210D9D6E954
:106710000201401AB060D6E90201884201D2B06895
:1067200000E0F068024641462846FFF74DFC5AE07B
:1067300095F8AA0200F01F0020B1012804D0022819
:1067400012D109E0002411E040F2AE20415D28465C
:10675000FFF737FC044609E040F2AE20415D2846D1
:10676000FFF72CFC044601E0002400BF00BF94B9F1
:1067700095F89C0203280ED105F52E7050F82400E0
:10678000006940B1C5F8D44205F52E7050F82400D8
:106790000169284688472846FFF76CFC23E007F08C
:1067A0007F012846FFF70AFC0446FF2C1BD0D4B912
:1067B00095F89C02032810D105F52E7050F824009E
:1067C000806950B1C5F8D44205F52E7050F8240008
:1067D00039468269284690478146B9F1000F02D0B8
:1067E0004846BDE8F0870020FBE7014600207047DF
:1067F00070B504460025012084F89C02D4F8B80244
:1068000038B12179D4F8B80242682046904700B1E7
:106810000325284670BD70B504460D462946D4F8B8
:10682000C802FBF72CFE70BD10B504462078002886
:106830002AD11648C0F8E044C4F8C8024FF0A0407E
:10684000124908600420087102211048C17100211A
:1068500081710221417200218172C17201738173C1
:10686000C173FCF761FA08B1FAF786F8802107488E
:10687000FBF717FD402200210448FBF717FD80229B
:1068800001210248FBF712FD002010BD681A00200C
:1068900010B50246D2F8C83201F08000802809D134
:1068A00001F07F0000EBC00403F1140000EB840052
:1068B000807810BD01F07F0000EBC00403F5157077
:1068C00000EB84008078F4E770B504460D4604F5CB
:1068D0002E70D4F8D41250F8210008B9032070BDEE
:1068E00094F89C02032811D104F52E70D4F8D41228
:1068F00050F82100006A48B104F52E70D4F8D41283
:1069000050F821002946026A204690470020E6E719
:1069100070B504460D4604F52E70D4F8D41250F824
:10692000210008B9032070BD94F89C02032811D1FE
:1069300004F52E70D4F8D41250F82100406A48B102
:1069400004F52E70D4F8D41250F821002946426A7A
:10695000204690470020E6E72DE9F04704460F4621
:1069600015461E464FF00008C1462B4632463946B2
:10697000D4F8C802FBF78EFD80464046FFF7D7FDEE
:1069800081464846BDE8F0872DE9F04704460D46AC
:1069900016461F464FF00008C1463B463246294680
:1069A000D4F8C802FBF7BDFD80464046FFF7BFFDA7
:1069B00081464846BDE8F08770B5044600250120B1
:1069C00084F89C020020C4F894026060C4F8A40219
:1069D00084F8A002D4F8B80258B1D4F8B8024068DC
:1069E00038B12179D4F8B80242682046904700B106
:1069F00003254023002211462046FFF7ADFF012169
:106A00004FF4B27001534021001F01514023002276
:106A100080212046FFF7A0FF0121A18440212162AF
:106A2000284670BD014691F89C02042803D191F8D4
:106A30009D0281F89C020020704710B5044694F82E
:106A40009C0203280BD1D4F8B80240B1D4F8B802A4
:106A5000C06920B1D4F8B802C16920468847002037
:106A600010BD02461174002070472DE9F041044624
:106A70000D46002600272946D4F8C802FCF77EFA06
:106A800006463046FFF753FD07463846BDE8F0811D
:106A900070B504460D46294604F2AA2000F07BF8A2
:106AA0000120C4F894024FF42C70005BC4F89802E3
:106AB00094F8AA0200F01F0020B1012809D0022892
:106AC00015D10DE004F2AA21204600F087F9064610
:106AD00016E004F2AA21204600F017FB06460FE05C
:106AE00004F2AA21204600F0D0F9064608E094F806
:106AF000AA0200F08001204600F005F8064600BF1B
:106B000000BF304670BD2DE9F04104460D46002619
:106B100000272946D4F8C802FBF726FD0646304672
:106B2000FFF705FD07463846BDE8F08170B504461D
:106B300000250026D4F8C802FCF743FA054628468B
:106B4000FFF7F5FC0646304670BD014691F89C0201
:106B5000042803D091F89C0281F89D02042081F85A
:106B60009C02002070472DE9F04704460D4616466A
:106B70001F464FF00008C1463B4632462946D4F82E
:106B8000C802FBF736FD80464046FFF7D0FC814641
:106B90004846BDE8F08770B505460E463446207875
:106BA0002870641C20786870641C2046FEF7ACF8DE
:106BB0006880641C641C2046FEF7A6F8A880641C4C
:106BC000641C2046FEF7A0F8E88070BD38B5044686
:106BD0000D46002000900DB9032038BDC4F8B8520E
:106BE00004F52E70D4F8D41250F82100C06A50B1C8
:106BF00004F52E70D4F8D42250F82200C16A6846F9
:106C00008847C4F8D002D4F8D802401CC4F8D8028F
:106C10000020E2E701460020704770B504460D46AB
:106C2000A88810BBE88800BB688880281DD2A87897
:106C300000F07F0694F89C02032804D129462046E0
:106C4000FFF7DAF915E084F89E6231462046FFF737
:106C50000CFF2046FFF70EFA1EB1022084F89C02BA
:106C600007E0012084F89C0203E029462046FFF754
:106C7000C3F970BD70B504460D460026D4F8B802BD
:106C800030B1D4F8B802294602682046904706463B
:106C9000304670BD70B504460E460025B0783D49BB
:106CA000087008460078012805D931462046FFF7CC
:106CB000A3F9032070BD94F89C02022802D0032897
:106CC00059D11FE033480078C0B132480078606085
:106CD000304801782046FFF7CDFF05463DB13146EB
:106CE0002046FFF789F9022084F89C0209E020463B
:106CF000FFF7C0F9032084F89C0202E02046FFF76A
:106D0000B9F943E02348007870B9022084F89C0266
:106D10002048007860601F4801782046FFF721F97D
:106D20002046FFF7A7F925E01A49097860688842EC
:106D30001DD021792046FFF714F9164800786060CD
:106D4000144801782046FFF795FF05465DB13146AE
:106D50002046FFF751F921792046FFF702F902207A
:106D600084F89C0206E02046FFF784F902E0204602
:106D7000FFF780F90AE031462046FFF73DF9054864
:106D800001782046FFF7EDF8032500BF00BF284635
:106D900090E700000001002070B505460C466088B1
:106DA000012805D1C5F8A4022846FFF763F90EE0D3
:106DB0006088022807D1A088001285F8A002284622
:106DC000FFF758F903E021462846FFF715F970BD93
:106DD00010B504462046FFF7A9FE10BD70B5044665
:106DE0000D460026287800F0600088B1202802D0E7
:106DF000402842D100E000BF04F52E70D4F8D41230
:106E000050F821002946826820469047064639E01E
:106E100068780A282AD2DFE800F01A24291F290AF4
:106E20000529150F29462046FFF7E5F923E02946F5
:106E30002046FFF7F2FE1EE029462046FFF72AFF14
:106E4000064618E029462046FFF7AAF913E029462E
:106E50002046FFF70BFB0EE029462046FFF79CFF7C
:106E600009E029462046FFF78AF804E02946204633
:106E7000FFF7C2F800BF00BF04E029462046FFF735
:106E8000BBF800BF00BF304670BD2DE9F047054696
:106E90000F464FF000093C79387800F06000F8B1F7
:106EA000202802D040287DD100E000BF214628469E
:106EB000FFF784F80646FF2E11D086B9C5F8D462D4
:106EC00005F52E7050F82600806840B105F52E704B
:106ED00050F826003946826828469047814610E1DE
:106EE000787800287AD001282FD003286ED195F821
:106EF0009C02022802D0032820D110E054B1802C3B
:106F000008D021462846FFF7FEFD80212846FFF7DE
:106F1000FAFD03E039462846FFF76EF813E078885B
:106F200040B93CB1802C05D0F88818B921462846D4
:106F3000FFF7E9FD2846FFF79DF804E039462846AB
:106F4000FFF75AF800BF00BFD4E095F89C02022872
:106F500002D003283BD110E054B1802C08D0214648
:106F60002846FFF7D0FD80212846FFF7CCFD03E03F
:106F700039462846FFF740F82EE0788820BB04F019
:106F80007F0018B121462846FFF704FB2846FFF78B
:106F900071F821462846FFF711F80646FF2E13D058
:106FA00096B900E0A8E0C5F8D46205F52E7050F857
:106FB0002600806840B105F52E7050F8260039464D
:106FC000826828469047814606E007E08DE0394612
:106FD0002846FFF711F800BF00BF8BE095F89C0230
:106FE000022802D0032879D126E034B1802C04D0C5
:106FF00039462846FFF700F875E004F08000802845
:1070000008D104F07F0000EB800105F1140000EBD3
:10701000810007E004F07F0000EB800105F5AA7015
:1070200000EB810080460020C8F8000002224146A3
:107030002846FFF70EF856E004F0800080280ED1B5
:1070400004F00F0000EB800105F1140000EB81005B
:10705000008A98B939462846FEF7CEFF43E004F08F
:107060000F0000EB800105F5AA7000EB8100008A9B
:1070700020B939462846FEF7BFFF34E004F080000F
:10708000802808D104F07F0000EB800105F1140096
:1070900000EB810007E004F07F0000EB800105F5C4
:1070A000AA7000EB810080460CB1802C03D1002037
:1070B000C8F800000CE021462846FFF7E9FB20B1A4
:1070C0000120C8F8000003E008E00020C8F8000034
:1070D000022241462846FEF7BCFF04E03946284616
:1070E000FEF78AFF00BF00BF04E039462846FEF7DE
:1070F00083FF00BF00BF04E039462846FEF77CFF4F
:1071000000BF00BF4846BDE8F0872DE9F0410546C5
:107110000E460027307800F0600030B1202802D001
:10712000402840D100E000BF00BF95F89C02012834
:1071300004D0022803D003282ED101E000BF00BFF5
:107140003079012823D831792846FEF73AFF0446E2
:10715000FF2C14D09CB905F52E7050F824008068DF
:1071600058B1C5F8D44205F52E7050F824003146C8
:10717000826828469047074602E0032700E003277D
:10718000F08840B93FB92846FEF774FF03E0314666
:107190002846FEF731FF04E031462846FEF72CFF73
:1071A00000BF00BF04E031462846FEF725FF00BFC0
:1071B00000BF3846BDE8F081704700000146014835
:1071C000704700004C1F002070B504460B46224655
:1071D0001978587801282CD140F61C0080581D7869
:1071E00005F00F060125B540ADB2284340F61C0559
:1071F000A85002F5106000EB4110006800F4004058
:10720000F0BB1889C0F30A001D7940EA854040EAC6
:10721000815040F0805040F4004002F5106505EBCD
:1072200041152D68284302F5106505EB41152860CE
:107230002DE040F61C0080581D7805F00F06012552
:10724000B540144E06EA0545284340F61C05A850F3
:1072500002F5306000EB4110006800F4004078B99E
:107260001889C0F30A001D7940EA854040F080503B
:1072700040F4004002F5306505EB41152D6800E053
:1072800005E0284302F5306505EB41152860002034
:1072900070BD00000000FFFF01460A464FF4106079
:1072A0008058C30ADB024FF41060835040F604009C
:1072B000805840F4807340F60400835000207047EB
:1072C0000FB470B504469DF81900012818D1A06BC1
:1072D00020F48030A063E0681B490840E060E0686B
:1072E00020F44010E0609DF82000012803D1E06800
:1072F00040F48010E060204600F028F8054613E0D6
:10730000E06840F04000E060204600F01FF80546CD
:107310009DF81D0020B9A06B40F48030A06303E00D
:10732000A06B20F48030A0639DF81600012807D1DF
:10733000A06840F00600A060A06840F02000A060B7
:10734000284670BC5DF814FBBFFFBDFF08B50146C1
:107350000020009000BF0098401C00900098B0F101
:10736000706F01D9032008BD086900F000400028B3
:10737000F1D000200090086940F00100086100BFD2
:107380000098401C00900098B0F1706F01D9032064
:10739000E9E7086900F001000028F1D100BFE2E749
:1073A00070B504460B46224619785878012848D112
:1073B00002F5106000EB4110006800F00040B0F1F1
:1073C000004F17D102F5106000EB4110006840F04B
:1073D000006502F5106000EB4110056002F51060D9
:1073E00000EB4110006840F0804502F5106000EBB2
:1073F0004110056040F63C0080581D7805F00F06EE
:107400000125B540ADB2A84340F63C05A85040F672
:107410001C0080581D7805F00F060125B540ADB25F
:10742000A84340F61C05A85002F5106000EB41107F
:1074300000682B4D284002F5106505EB41152860CA
:107440004BE002F5306000EB4110006800F00040B6
:10745000B0F1004F17D102F5306000EB4110006829
:1074600040F0006502F5306000EB4110056002F568
:10747000306000EB4110006840F0804502F530605C
:1074800000EB4110056040F63C0080581D7805F087
:107490000F060125B540134E06EA0545A84340F600
:1074A0003C05A85040F61C008558187800F00F06DF
:1074B0000120B0400B4E06EA0040854340F61C0018
:1074C000855002F5306000EB41100068064D284001
:1074D00002F5306505EB41152860002070BD000005
:1074E000007833EC0000FFFF0078F3EF01460A4616
:1074F000D2F8000E20F00300C2F8000E40F604009F
:10750000805820F0020340F60400835000207047AA
:1075100001460A46D2F8000E20F00300C2F8000E21
:1075200040F60400805840F0020340F60400835007
:10753000002070470FB4F0B5054600272E46002402
:1075400005E0002105F5827040F82410641C0F2C22
:10755000F7D39DF82200A0B940F60400805940F00E
:10756000020140F604008151A86B40F40010A863AA
:10757000A86B20F40020A863A86B20F48020A863E7
:1075800007E0A86B20F40010A863A86B40F400206B
:10759000A8630020C6F8000E9DF81D0001280CD13C
:1075A0009DF81B0020B90021284600F00AFD08E0E4
:1075B0000121284600F005FD03E00321284600F0E4
:1075C00000FD1021284600F002FC00B101272846EA
:1075D00000F0D5FB00B1012700214FF4016081517B
:1075E000001D815140F61C00815100242EE006F55B
:1075F000106000EB4410006800F00040B0F1004F54
:1076000010D13CB94FF0006106F5106000EB44105A
:1076100001600DE04FF0904106F5106000EB441062
:10762000016005E0002106F5106000EB44100160E8
:10763000002106F5106000EB441001614FF67F3128
:1076400006F5106000EB44108160641C9DF8180082
:10765000A042CCD800242EE006F5306000EB4410A8
:10766000006800F00040B0F1004F10D13CB94FF07D
:10767000006106F5306000EB441001600DE04FF052
:10768000904106F5306000EB4410016005E00021F8
:1076900006F5306000EB44100160002106F5306013
:1076A00000EB441001614FF67F3106F5306000EBCE
:1076B00044108160641C9DF81800A042CCD84FF49F
:1076C0000160805920F480714FF4016081510020E5
:1076D000A8616FF0804068619DF81A0018B9A86928
:1076E00040F01000A861A8690A490843A8619DF804
:1076F0001E0018B1A86940F00800A8619DF822009A
:10770000012803D1A86904490843A8613846F0BCA0
:107710005DF814FB00383C80040000400146886896
:1077200020F00100886000207047000070B503461B
:107730000C4619461D6C1848854209D94FF4306033
:10774000405800F00040B0F1004F01D1002070BD62
:107750000026C1F8106BD1F8100B40F40026C1F8D8
:10776000106BD1F8100B40F01806C1F8106BD1F86F
:10777000100B40F0C046C1F8106B012C09D1C1F8C4
:10778000142B4FF43060405840F080264FF43060A6
:1077900046500020DBE700000A30544F30B5044665
:1077A0000B4622461978587801281ED102F5106040
:1077B00000EB4110006820F4001502F5106000EBAA
:1077C000411005601879032802D0187902282AD1BF
:1077D00002F5106000EB4110006840F0805502F5A2
:1077E000106000EB411005601DE002F5306000EB19
:1077F0004110006820F4001502F5306000EB4110E4
:1078000005601879032802D0187902280BD102F5F7
:10781000306000EB4110006840F0805502F53060A8
:1078200000EB41100560002030BD30B504460B462A
:10783000224619785878012821D102F5106000EB12
:107840004110006800F0004060B959B102F51060C5
:1078500000EB4110006820F0804502F5106000EB5D
:107860004110056002F5106000EB4110006840F423
:10787000001502F5106000EB4110056020E002F5F4
:10788000306000EB4110006800F0004060B959B171
:1078900002F5306000EB4110006820F0804502F5F1
:1078A000306000EB4110056002F5306000EB4110E4
:1078B000006840F4001502F5306000EB41100560EF
:1078C000002030BD2DE9F84381460E4690464D46D6
:1078D0003478707801287DD1306920BB05F51060BF
:1078E00000EB44100069E649084005F5106101EB22
:1078F0004411086105F5106000EB4410006940F484
:10790000002105F5106000EB4410016105F51060E1
:1079100000EB44100069C10CC90405F5106000EBD0
:10792000441001616FE005F5106000EB4410006940
:10793000C10CC90405F5106000EB4410016105F5A8
:10794000106000EB44100069CD49084005F5106156
:1079500001EB4411086194B9B1683069884201D9DA
:10796000B068306105F5106000EB4410006940F428
:10797000002105F5106000EB4410016135E0B168AD
:1079800030690844401EB0FBF1F087B205F5106085
:1079900000EB44100069BA49C94301EAC7410843F2
:1079A00005F5106101EB44110861307901281CD103
:1079B00005F5106000EB4410006920F0C04105F5AA
:1079C000106000EB4410016105F5106000EB4410FD
:1079D000006900E099E04FF0C04101EA47710843B7
:1079E00005F5106101EB4411086105F5106000EB2D
:1079F000441000693169C1F31201084305F51061B3
:107A000001EB44110861B8F1010F36D1F06928B1DA
:107A100005F5106000EB4410F169416130790128EF
:107A20001ED140F60800405900F4807060B905F599
:107A3000106000EB4410006840F0005105F5106044
:107A400000EB441001600BE005F5106000EB441002
:107A5000006840F0805105F5106000EB44100160B3
:107A600005F5106000EB4410006840F0044105F596
:107A7000106000EB44100160FEE005F5106000EBC3
:107A80004410006840F0044105F5106000EB44101C
:107A90000160307901280FD030690028ECD040F621
:107AA00034004059317801F00F0201219140084320
:107AB00040F634014851DFE040F60800405900F438
:107AC000807060B905F5106000EB4410006840F06C
:107AD000005105F5106000EB441001600BE005F566
:107AE000106000EB4410006840F0805105F5106014
:107AF00000EB44100160CDF80080308A83B2327808
:107B00004846F16800F0DAFAB6E005F5306000EBBF
:107B100044100069C10CC90405F5306000EB441045
:107B2000016105F5306000EB4410006954490840DC
:107B300005F5306101EB4411086104BB306908B1FF
:107B4000B0683061B068306205F5306000EB441019
:107B50000069316AC1F31201084305F5306101EB98
:107B60004411086105F5306000EB4410006940F4F1
:107B7000002105F5306000EB4410016143E03069FD
:107B8000D0B905F5306000EB44100069B168C1F36D
:107B90001201084305F5306101EB4411086105F558
:107BA000306000EB4410006940F4002105F53060BE
:107BB00000EB4410016126E0B16830690844401EC2
:107BC000B0FBF1F087B2B0687843306205F5306001
:107BD00000EB441000692A49C94301EAC741084340
:107BE00005F5306101EB4411086105F5306000EBEB
:107BF00044100069316AC1F31201084305F5306190
:107C000001EB44110861B8F1010F07D1F06828B108
:107C100005F5306000EB4410F168416130790128CE
:107C20001ED140F60800405900F4807060B905F597
:107C3000306000EB4410006840F0005105F5306002
:107C400000EB441001600BE005F5306000EB4410E0
:107C5000006840F0805105F5306000EB4410016091
:107C600005F5306000EB4410006840F0044105F574
:107C7000306000EB441001600020BDE8F883000094
:107C8000FFFF07E078B503460024009400201A4661
:107C90004C78012C35D10C7802F5106505EB4414B5
:107CA000246804F00044B4F1004F60D10C7805EB77
:107CB0004414246844F000660C7805EB44142660F4
:107CC0000C7805EB4414246844F080460C7805EBEE
:107CD0004414266000BF009C641C009442F210759E
:107CE000009CAC4201D901200AE00C7802F5106535
:107CF00005EB4414246804F00044B4F1004FEAD0CA
:107D000035E00C7802F5306505EB4414246804F086
:107D10000044B4F1004F2AD10C7805EB44142468D8
:107D200044F000660C7805EB441426600C7805EBF3
:107D30004414246844F080460C7805EB4414266013
:107D400000BF009C641C009442F21075009CAC4281
:107D500001D901200AE00C7802F5306505EB4414E6
:107D6000246804F00044B4F1004FEAD000BF78BDAD
:107D70000146886840F0010088600020704708B51F
:107D800001460020009000BF0098401C0090009821
:107D9000B0F1706F01D9032008BD086900F0004000
:107DA0000028F1D0002000901020086100BF00984A
:107DB000401C00900098B0F1706F01D90320EBE7F0
:107DC000086900F010001028F1D00020E4E708B5A1
:107DD00002460020009000BF0098401C00900098D0
:107DE000B0F1706F01D9032008BD106900F00040A8
:107DF0000028F1D000200090202040EA811010617E
:107E000000BF0098401C00900098B0F1706F01D93D
:107E10000320E9E7106900F020002028F1D00020BD
:107E2000E2E710B501460B4640F60804E45804F0BA
:107E300006020AB9002006E0022A01D0062A01D172
:107E4000022000E00F2010BD0146486900F001004B
:107E5000704701460B4640F61800C258001DC05836
:107E6000024090B2704701460B4640F61800C258D7
:107E7000001DC0580240100C704770B502461346F2
:107E80004FF40166F45840F63406F55801F00F0639
:107E900025FA06F606F0010644EAC61403F5106654
:107EA00006EB4116B66806EA040070BD10B502463E
:107EB000134603F5306404EB4114A06840F6140443
:107EC000E458204010BD014648698A691040704757
:107ED0002DE9F04104460D46274628464FEA920C0C
:107EE00002F0030300210AE04FF4805858F807809D
:107EF000C0F80080401C401C401C401C491C6145CF
:107F0000F2D39BB100214FF4805858F8076000BFAE
:107F10004FEAC10826FA08F880F80080491C401C86
:107F2000A3F101081FFA88F3002BF1D1BDE8F0811D
:107F300070B504460E460025E06820F0C040E060C1
:107F4000012E10D1E06840F00050E06000BF0A2030
:107F5000F9F7ACFF0A352046FFF776FF012815D068
:107F6000C82DF4D312E07EB9E06840F08040E060B4
:107F700000BF0A20F9F79AFF0A352046FFF764FF91
:107F800020B1C82DF5D301E0012070BDC82D01D16D
:107F90000120FAE70020F8E710B502460B4611462B
:107FA000D1F8000820F4FE60C1F80008D1F80008FC
:107FB0004FF4FE6404EA03142043C1F800080020D3
:107FC00010BD02461346D3F800080843C3F8000862
:107FD0000020704730B503461446022C49D12D4885
:107FE000814204D32C48814201D20F2245E02A4825
:107FF000814204D32948814201D20E223DE0274824
:10800000814204D32648814201D20D2235E0244822
:10801000814204D32348814201D20C222DE0214821
:10802000814204D32048814201D20B2225E01E4820
:10803000814204D31D48814201D20A221DE01B481F
:10804000814204D31A48814201D2092215E018481E
:10805000814204D31748814201D208220DE015481D
:10806000814204D31448814201D2072205E006224E
:1080700003E00CB9092200E00922D86820F470500E
:10808000D860D8684FF4705505EA82252843D86037
:10809000002030BDC0ACD800C0E1E4000024F400F2
:1080A00080730601A0491A01002D310140A44C0142
:1080B00000366E0120ABA6010048E8012DE9F0432F
:1080C00004460D461E46DDF81CC0A0462946BCF1FC
:1080D000000F12D1F01C870800230CE0D1F80090AB
:1080E00008F5805000EB0230C0F80090491C491C94
:1080F000491C491C5B1CBB42F0D30020BDE8F08347
:1081000000BFFEE700B587B01B4B6A4601211B4844
:10811000F8F790FF0098A0F2092050BB1648C078ED
:1081200000061549897840EA01401349497840EA38
:10813000012011490978084300EE100AB8EEC00A80
:108140000F4880ED000A0C48C07900060A49897979
:1081500040EA01400849497940EA01200649097985
:10816000084300EE100AB8EEC00A054880ED010A87
:1081700000BF00BF07B000BDC001002034020020D6
:10818000B801002002480068C0F3022070470000D8
:108190000CED00E010B5002804DB0A07130E054AB9
:1081A000135406E00A07140E034A00F00F031B1FC6
:1081B000D45410BD00E400E018ED00E0EFF30580BA
:1081C0007047000000B58BB0012009900020079097
:1081D00001200890002001900290039004900690E6
:1081E000059001A90C48F8F775FE0B48F9F714FB48
:1081F00002210948F8F7B4FD0E200A90069001A963
:108200000648F8F767FE0548F9F706FB1021034812
:10821000F8F7A6FD0BB000BD0C02002034020020D0
:1082200010B5044A06210020F8F71AFAFFF7CAFF32
:1082300010BD00004D09000810B52DED048BBD48A0
:108240000068A0F2012007287ED2DFE800F00405D4
:10825000060708090A0000BF00BF00BF00BF00BF3B
:1082600000BFB4480078401EB3490870B34809788D
:1082700000EB41104069322825D8B048AE49097852
:1082800000EB41104069401CAC49AB4A127801EB4D
:1082900042114861AA484078A949097840EA01207A
:1082A000A649A54A127801EB42110880A348A249C9
:1082B000097800EB41100088A0499F4A127801EB31
:1082C000421108822FE19D489B49097800EB41103B
:1082D000008800B29949984A127801EB421108814E
:1082E000974840789649097840EA01209349924A94
:1082F000127801EB421108809148C0789049897842
:1083000040EA012000B28D498B4A127801EB4211FC
:1083100048808B4840798A49097940EA012001B2B6
:108320008648854A127800EB421081808448807923
:108330008249814A127801EB4211C8807F487E4908
:10834000097800EB411000E0EEE000887B497A4AB2
:10835000127801EB4211B1F90810401AB0F5805FB4
:108360000EDD76487449097800EB41104089401EC3
:1083700001B27248704A127800EB421041811EE04F
:108380006E486D49097800EB411000886B496A4AD4
:10839000127801EB4211B1F90810401A10F5805F14
:1083A0000DDA66486449097800EB41104089401CA9
:1083B00001B26248604A127800EB421041815F4886
:1083C0005D49097800EB4110007F01282AD15B4903
:1083D000594A127801EB42110A885849564B1B78CA
:1083E00001EB4311B1F90A1002EB4131534A524BF0
:1083F0001B7802EB4312128A881A02F050FE41ECFD
:10840000190B9FED500B53EC102B02F05FFE41EC6B
:10841000180B02F015FE4949474A127801EB421148
:10842000C8605CE045484449097800EB4110007F92
:1084300002282AD14149404A127801EB42110A88A8
:108440003E493D4B1B7801EB4311B1F90A1002EB99
:1084500041323A49384B1B7801EB4311098A501AD3
:1084600002F01DFE41EC190B9FED380B53EC102B65
:1084700002F02CFE41EC180B02F0E2FD2F492E4ACF
:10848000127801EB4211C86029E02C492A4A12787F
:1084900001EB42110A882949274B1B7801EB431154
:1084A000B1F90A1002EB41322449234B1B7801EB4E
:1084B0004311098A501A02F0F2FD41EC190B9FEDAD
:1084C000250B53EC102B02F001FE41EC180B02F0CF
:1084D000B7FD1A49184A127801EB4211C8601748D3
:1084E0001549097800EB4110C0684FF4B47190FB56
:1084F000F1F000B21149104A127801EB42110883E1
:108500000E480D49097800EB4110C0684FF4B47172
:1085100090FBF1F201FB120000B20849064A127802
:1085200001EB4211488300E000BF00BFBDEC048BAB
:1085300010BD0000FC6B0020B4010020146B002073
:10854000A8010020841C12AEC8BF623F01280005AC
:10855000A000543F012DA005B480A63F10B50246EF
:10856000002009E012F8013B4340DBB2054C34F82F
:10857000233083EA202398B20B1EA1F10101F1D12F
:1085800010BD000018B300082DE9F04707463E462D
:1085900056B900BF502080F31188BFF34F8FBFF34F
:1085A0006F8F00BF00BFFEE717480068864201D109
:1085B000002426E001F0F0F975691448D0F8008035
:1085C0001348D0F8009001F011FA454501D04D450F
:1085D00001D1022415E00F4885420BD1B06A38B9A9
:1085E00096F85800012801D102240AE0032408E08B
:1085F000022406E00848854200D00DB9042400E0BA
:1086000001242046BDE8F08780000020840000207F
:10861000880000205C26002048260020014601EB4F
:108620004100024A02EB401070470000186C002025
:108630000146024800EB411070470000146B002017
:1086400010B5144890ED020AF0EE400A9FED122A90
:10865000DFED121AB2EE041A9FED110A0022114644
:108660001048F8F775FA0B4890ED020AF0EE400A50
:108670009FED092ADFED091AB2EE041A9FED080AF0
:10868000002211460848F8F763FA012000F080F94B
:1086900010BD0000A06D00206F12033C8FC2F53D9D
:1086A00000000000A40200209403002010B5F8F799
:1086B00067F9002452E0E0B2FFF7B0FF294941F822
:1086C00024009FED290A01F1080000EB840080EDF1
:1086D000000A9FED250A01F1100000EB840080EDF7
:1086E000000A9FED212ADFED201A9FED1F1ADFED12
:1086F0001E0A9FED1D0A002221461C48F8F728FAA1
:10870000184850F8240090ED080A1648103000EB85
:10871000840080ED000A4FF4FA60F9F7C7FB9FED83
:10872000122ADFED111A9FED101ADFED0F0A9FEDEF
:108730000E0A002221460D48F8F70AFA094850F8B7
:10874000240090ED080A0748103000EB840080ED0B
:10875000000A4FF4FA60F9F7A9FB641C022CAADBAB
:1087600010BD0000A06D0020000000009403002058
:10877000F9F7C2FCFCF7E4FAFBF7FAFEFBF798FE08
:10878000FBF752FEFBF772FEFBF77AFFFBF7D0FF19
:10879000FBF7EAFFFCF708F800F080F9FBF7CCFEE6
:1087A00000F0AEF900BFFEE710B50020FFF740FF74
:1087B0000A490860DFED0A0A9FED0A0A0A4A002109
:1087C0000A48FCF771FADFED0A0A9FED0A0A0A4A25
:1087D00000210A48FCF768FA10BD0000D40100200F
:1087E00000007A4400803B45D8010020006D002045
:1087F0000000FA4400C0DA45E4010020486D002082
:1088000010B52DED028BB0EE408A0C480068B0F92F
:10881000020000EE900AF8EEE00AB0EE600AF0EE18
:10882000480A0748FCF748F9BDEEC00A10EE100AE6
:1088300000B204490880BDEC028B10BDD4010020B9
:10884000006D0020FC01002011B52DED020B81B060
:108850000446102C05D0202C03D04FF0FF3004B07C
:1088600010BD122040EA44101349086000208860BF
:10887000C860082008619DF80400104908709DF840
:10888000050048709DF8060088709DF80700C870C4
:108890009DF8080008719DF8090048719DF80A00CC
:1088A00088719DF80B00C8716B460A46024904485E
:1088B000F8F76BFA0020D2E7E86C0020C80100202E
:1088C0003402002038B50446102C04D0202C02D0ED
:1088D0004FF0FF3038BD092040EA44100D490860D0
:1088E000002088600220C8600820086110200A4922
:1088F0000870002048708870C870087148718871CD
:10890000C8716B460A4603490448F8F73EFA00204E
:10891000E0E70000E86C0020C801002034020020DD
:1089200011B52DED020B81B00446102C05D0202C82
:1089300003D04FF0FF3004B010BD0C2040EA4410CB
:108940001049086000208860C860082008619DF810
:1089500004000D4908709DF8050048709DF8060058
:1089600088709DF80700C8700020087148718871F0
:10897000C8716B460A4603490448F8F706FA002016
:10898000D9E70000E86C0020C80100203402002074
:1089900070B50546FFF712FC10B16FF0050404E056
:1089A000002415B1284601F01DF9204670BD0000D5
:1089B000F8B505460E462F4617B106F07F4010B1B8
:1089C0006FF003041EE0FFF7F9FBB0B10020009048
:1089D0006A463146384601F08BFB10B96FF002044D
:1089E00010E03446009868B14FF0805006490860A6
:1089F000BFF34F8FBFF36F8F04E03146384601F06D
:108A00000FFB04462046F8BD04ED00E02DE9F84FC9
:108A100080460D4616461F46C346BBF1000F02D0E6
:108A200005F07F4010B16FF0030434E0FFF7C6FBA0
:108A300010B16FF005042EE006F0010010B14FF008
:108A4000010901E04FF0000906F0020010B14FF0FB
:108A5000000A01E04FF0010A4B46524629465846AB
:108A6000009701F057FB044606F0010050B105EAFB
:108A70000400A8420FD017B16FF001040BE06FF0B3
:108A8000020408E005EA040028B917B16FF00104F8
:108A900001E06FF002042046BDE8F88F10B5FFF743
:108AA0008DFB10B16FF0050409E00648006820B99D
:108AB000012004490860002401E04FF0FF34204603
:108AC00010BD0000D000002010B5FFF777FB10B1FB
:108AD0006FF0050412E002F043F820B1012809D03C
:108AE000022806D101E0012407E001F03DFA00244C
:108AF00003E000BF4FF0FF3400BF00BF204610BDB1
:108B000070B5FFF75BFB10B16FF005041FE0114873
:108B10000068012819D100BF801F0021002804DB54
:108B20000A07130E0C4A135406E00A07150E0B4AE7
:108B300000F00F031B1FD55400BF00BF02200549E2
:108B4000086001F0B5F9002401E04FF0FF34204641
:108B500070BD0000D000002000E400E018ED00E04F
:108B600010B5FFF72BFB10B16FF0050418E001F012
:108B7000F7FF20B101280FD002280CD109E0012411
:108B800002F044F9012803D001F0EAFF00B9A41E65
:108B900005E0002403E000BF4FF0FF3400BF00BF3A
:108BA000204610BD10B501F0D5FF0446204610BD8B
:108BB0002DE9FF4780468946144600200390FFF7C1
:108BC000FDFA00284ED1B8F1000F4BD080261825B1
:108BD0008246471E44B3206808B1D4F800A0A069BB
:108BE00000B1A5692DB1382D03D8207900F001001E
:108BF00018B1002004B0BDE8F087606908B1606971
:108C00008608A06840B1E0685C2805D3206918B1E7
:108C1000606908B1012708E0A06830B9E06820B9B0
:108C2000206910B9002700E00027012F0CD121692D
:108C3000A0684B463246CDE900510290514640466D
:108C400001F02AFF03900DE067B903A8B2B24B46CA
:108C50005146CDE90050404601F0ECFE012801D01C
:108C6000002003900398C5E72DE9F04106463746FA
:108C7000FFF7A4FA10B16FF0050410E017B96FF018
:108C800003040CE03846FFF77FFC0546042D04D0B2
:108C90000024384600F0D4FF01E06FF002042046C3
:108CA000BDE8F0812DE9F04105460E4619480768F8
:108CB00000201949096881F85A0017480068001D0A
:108CC00000F0F2FD681C38B936B113480168091D7F
:108CD000124800F055FE1AE07C190F480068446005
:108CE000BC4207D20C480168091D0D48006800F01D
:108CF0002DFE0CE008480168091D0A48006800F0D4
:108D000025FE09480068844201D207480460BDE896
:108D1000F081000094000020800000205C260020EC
:108D20008800002084000020B000002010B5044618
:108D300000F032FE24480068401C234908602348A4
:108D4000006840B9214804600846006801280DD138
:108D500000F0FEF90AE01E48006838B91B480068B8
:108D6000C06AE16A884201D818480460194800685E
:108D7000401C184908600846006860641649E06AAB
:108D80000968884202D91449E06A0860E16A01EB87
:108D90008101124A02EB8100211D00F0F1FD00F07B
:108DA00025FE0B48006868B108480068C06AE16A9F
:108DB000884207D24FF0805009490860BFF34F8FB7
:108DC000BFF36F8F10BD00009000002080000020D6
:108DD0009C000020AC00002098000020AC21002066
:108DE00004ED00E008B500F0D7FD12480068E8B9CE
:108DF000114800F09BFD114800F098FD0E48104905
:108E000008600E480F49086000200F4B0F4A1021E0
:108E100000900A2001F0F8FA064908600846006848
:108E200020B10BA10348006800F0A0FE00F0DEFDB9
:108E300008BD0000C4000020702600208426002009
:108E4000BC000020C000002098260020E82600205A
:108E5000546D72510000000010B516E000F09CFD4A
:108E60000C48C068C468201D00F01EFD0A48006858
:108E7000401E0949086009480068401E074908600B
:108E800000F0B4FD204600F05FF8044800680028B8
:108E9000E4D110BD48260020900000208C00002066
:108EA00070B504460D46206C70B1216CE068014439
:108EB000E160D4E90210884201D32168E1602846CC
:108EC000226CE168F7F7C7FA70BD2DE9F04104465E
:108ED0000F4615464FF00008A66B206C48B9206875
:108EE00000282CD1A06801F0F3FE80460020A0608D
:108EF00025E07DB93946226C6068F7F7ACFA216C41
:108F0000606808446060D4E90101884217D3206892
:108F1000606014E03946226CE068F7F79CFA216C37
:108F2000E068411AE1602168E068884203D2216C60
:108F3000A068411AE160022D01D106B1761E701CB5
:108F4000A0634046BDE8F08110B5044694F859008E
:108F500030B9206B00F068FD204600F065FD1AE096
:108F600094F85900012803D1204600F05DFD12E07D
:108F700094F85900022801D1012000E0002050B9E6
:108F800000BF502080F31188BFF34F8FBFF36F8F66
:108F900000BF00BFFEE710BD0146084A1268126814
:108FA0000AB9012200E000220A600A6822B9034AD5
:108FB0001268D268106800E000207047BC000020F2
:108FC00030B54FF47053174800F007042CB1C01DA2
:108FD00020F00700134C041B1B1B0246124C22609E
:108FE0000024114D6C60D018083820F007000F4C99
:108FF000206000240D4D2D686C600C4D2D682C6098
:109000001146441A4C60094C24680C60084D4C68A9
:109010002C60084D4C682C604FF00044064D2C60CD
:1090200030BD0000402E0020D4000020DC000020D5
:10903000E4000020E0000020F000002000BFFFF767
:109040000BFF064800680128F9D94FF08050044909
:109050000860BFF34F8FBFF36F8FF0E7AC210020A4
:1090600004ED00E02DE9F04106460D46174698460E
:10907000069C0DB9246000E02760E66325640121A9
:10908000204601F031FA84F84C80BDE8F0812DE9EA
:10909000F05F82460E4690469B460A9F0C9C4FEA24
:1090A0008801A522206BF7F71BFAA8F10100216BBC
:1090B00001EB800929F0070909F0070008B9012030
:1090C00000E0002050B900BF502080F31188BFF3AA
:1090D0004F8FBFF36F8F00BF00BFFEE786B1002543
:1090E00007E0715D04F134004155705D00B902E0A4
:1090F0006D1C102DF5D300BF00214320015502E067
:10910000002084F83400382F00D33727E762E76463
:1091100000202065201D00F016FC04F1180000F06E
:1091200012FC2461C7F13800A06164620020606510
:1091300084F8580084F85A005A465146484600F0D0
:1091400081FB20600B9808B10B980460BDE8F09F8C
:1091500010B5002407E004EB84010F4A02EB810004
:1091600000F0E4FB641C382CF5D30C4800F0DEFB67
:109170000B4800F0DBFB0B4800F0D8FB0A4800F07E
:10918000D5FB0A4800F0D2FB0448094908600448AE
:109190000849086010BD0000AC2100200C2600200A
:1091A0002026002034260020482600205C260020AF
:1091B000840000208800002010B50146164800E019
:1091C000006803688B42FBD30246436813448B421A
:1091D00004D143684C682344436001460A464B6807
:1091E00013440468A34211D10C4C03682468A342C1
:1091F00008D04B680468646823444B6003681B68AC
:109200000B6005E0054B1B680B6001E003680B6019
:10921000884200D0016010BDD4000020DC00002096
:109220002DE9F04104460D4616461F464FF0000852
:1092300065602461B5420CD8F01BA169884202D355
:109240004FF0010811E0211D0948006800F07EFB85
:109250000BE0BE4204D2BD4202D34FF0010804E04D
:10926000211D0448006800F071FB4046BDE8F08114
:10927000C0000020BC00002070B5054600F08CFB4B
:10928000A86B08B9012400E0002400F0AFFB2046E1
:1092900070BD70B5054600F07FFBA86BE96B884296
:1092A00001D1012400E0002400F0A0FB204670BDA5
:1092B000F8B505460F461A480068C068C468201D06
:1092C00000F0F2FA94F8280000F00400E8B1A06978
:1092D00041192B463A462046FFF7A2FFD8B100209D
:1092E00003462A4601460090204601F04DFE064600
:1092F00056B900BF502080F31188BFF34F8FBFF3E2
:109300006F8F00BF00BFFEE705E094F8280020F053
:10931000010084F828002046216A8847F8BD000033
:10932000BC000020F0B587B0A0E00398002811DA57
:1093300004AE56B900BF502080F31188BFF34F8FA1
:10934000BFF36F8F00BF00BFFEE7D6E90020B16812
:10935000904700BF03980028E6DB059C606908B9C8
:10936000012000E0002010B9201D00F09DFA02A8A5
:1093700000F0DEF8054603980A2875D2DFE800F011
:1093800009050739416306083A4200BF00BF00BF24
:1093900000BF94F8280040F0010084F828000498E9
:1093A000A269811803462A462046FFF739FFF8B123
:1093B0002046216A884794F8280000F00400B8B1DC
:1093C000002000900498A169421800231946204605
:1093D00001F0DAFD074657B900BF502080F311882D
:1093E000BFF34F8FBFF36F8F00BF00BFFEE700BF1B
:1093F0003BE000BF94F8280020F0010084F828002A
:1094000033E000BF94F8280040F0010084F8280001
:109410000498A061A06908B1012000E0002050B9C3
:1094200000BF502080F31188BFF34F8FBFF36F8FC1
:1094300000BF00BFFEE7A06941192B462A4620461F
:10944000FFF7EEFE11E094F8280000F0020018B9D2
:10945000204600F0E9FA05E094F8280020F0010029
:1094600084F8280001E0FFE700BF00BF002203A945
:109470000448006801F0D6F900287FF456AF07B021
:10948000F0BD0000C4000020F8B505460C4600F011
:109490006BFD684600F04CF80646009820BB44B9C6
:1094A000B54206D801F0B2FC31462846FFF700FF6E
:1094B0001CE03CB10E480068006808B9012000E0DB
:1094C00000200446A91B22460A48006800F064FBFD
:1094D00001F09CFC50B94FF0805007490860BFF381
:1094E0004F8FBFF36F8F01E001F090FCF8BD0000DB
:1094F000C0000020C400002004ED00E00A49096813
:10950000096809B9012100E0002121B14FF0FF31C4
:10951000064A116006E004490968C968C868034A38
:10952000416811607047000084000020B0000020F6
:1095300070B5044601F024FB0546074800688542E3
:1095400004D200F00BF80120206001E00020206030
:1095500001480560284670BDCC0000202DE9F84385
:1095600034E025480068C068056823480068C06882
:10957000C468201D00F098F92046216A884794F8B5
:10958000280000F0040008B3A0694619AE4207D9CC
:1095900066602461211D1848006800F0D7F915E0C5
:1095A000002003462A4601460090204601F0ECFCCC
:1095B000074657B900BF502080F31188BFF34F8F83
:1095C000BFF36F8F00BF00BFFEE700BF0A4800680F
:1095D000006808B9012000E000200028C1D006483A
:1095E000D0F8008005480068034908600348C0F8C7
:1095F0000080BDE8F8830000BC000020C00000200F
:109600000E480068401C08B9012000E0002050B955
:1096100000BF502080F31188BFF34F8FBFF36F8FCF
:1096200000BF00BFFEE700BF502080F31188BFF3EA
:109630004F8FBFF36F8F00BF00BFFEE7F400002025
:1096400010B50346002022B903EA010434B1012019
:1096500004E003EA01048C4200D1012010BD08B5EA
:1096600000BF6846FFF798FC044620460099FFF7C4
:109670000BFFFFF757FEF4E770B5044600F08CF9D6
:1096800094F9455010E0606A08B9012000E000201C
:1096900038B904F1240001F06DFB18B100F040FB73
:1096A00000E003E0681E45B2002DECDC00BFFF20A7
:1096B00084F8450000F09AF900F06EF994F94450EE
:1096C00010E0206908B9012000E0002048B904F149
:1096D000100001F04FFB08B100F022FB681E45B2FC
:1096E00000E001E0002DECDC00BFFF2084F8440026
:1096F00000F07CF970BD00002DE9F04104464FF008
:10970000000800F031FC4948006808B9FFF758FC30
:10971000474800682040002870D1D4B1083404F0D4
:109720000700B0B104F00700C0F10800044404F0E1
:10973000070008B9012000E0002050B900BF502008
:1097400080F31188BFF34F8FBFF36F8F00BF00BF4F
:10975000FEE7002C52D03748006884424ED8364E7F
:109760003046056801E02E462D686868A04202D2A6
:1097700028680028F7D12D48006885423ED030681F
:1097800000F10808286830606868001B102819D9A3
:109790002F1907F0070008B9012000E0002050B998
:1097A00000BF502080F31188BFF34F8FBFF36F8F3E
:1097B00000BF00BFFEE76868001B78606C60384639
:1097C000FFF7FAFC1B4968680968081A194908601C
:1097D0000846006819490968884203D2154800689C
:1097E00016490860124968680968084368600020E3
:1097F000286013480068401C1149086001F006FB0E
:1098000008F0070008B9012000E0002050B900BFAF
:10981000502080F31188BFF34F8FBFF36F8F00BFCD
:1098200000BFFEE74046BDE8F0810000DC000020FC
:10983000F0000020E0000020D4000020E400002020
:10984000E8000020001F4FF080730360001F21F02C
:1098500001030360001F054B036014380260001F02
:109860006FF0020303602038704700000196000883
:1098700010B5F2EE040AB2EE040A1020FEF7E4FF7F
:10988000034890ED000A1020FFF74AF810BD0000D1
:109890000002002010B50446102202492046FAF7C3
:1098A000A3FC10BDD86C002001460A69D1E9013043
:1098B0009860D1E9010358605068884201D18868F6
:1098C0005060002008611068401E106010687047EA
:1098D00005490968886904490968C96AC1F13801FC
:1098E000014A12689161704780000020034B0360B9
:1098F000034B0B6080231360704700008827002013
:10990000E4270020034B0360034B0B604FF480738C
:1099100013607047E4290020402A002070B50446F7
:109920000D462946204600F07BFB70BD00F1080182
:1099300041604FF0FF31816000F10801C1600161B9
:1099400000210160704700210161704710B5024697
:109950000B685C1C0CB9106907E002F1080000E01C
:109960004068446824689C42FAD944684C604C685A
:10997000A160886041600A611468641C146010BDB5
:1099800042684A6093688B6093685960916008618F
:1099900003685B1C0360704700BF502080F3118890
:1099A000BFF34F8FBFF36F8F00BF0E480068401C9E
:1099B0000C49086008460068012812D10A4800686E
:1099C000C0B208B9012000E0002050B900BF50200B
:1099D00080F31188BFF34F8FBFF36F8F00BF00BFBD
:1099E000FEE77047F400002004ED00E00D48006839
:1099F00050B900BF502080F31188BFF34F8FBFF3E1
:109A00006F8F00BF00BFFEE706480068401E054993
:109A100008600846006820B9002080F3118800BF64
:109A200000BF7047F400002070B506463546002E92
:109A300044D0083D2C46224960680968084008B1B6
:109A4000012000E0002050B900BF502080F31188B1
:109A5000BFF34F8FBFF36F8F00BF00BFFEE72068DB
:109A600008B9012000E0002050B900BF502080F369
:109A70001188BFF34F8FBFF36F8F00BF00BFFEE7AA
:109A80000F49606809680840C0B12068B0B90C4946
:109A9000606809688843606000F066FA0949606898
:109AA00009680844074908602046FFF785FB064817
:109AB0000068401C0449086001F0A8F970BD00006E
:109AC000F0000020E0000020EC00002000204FF01B
:109AD000E02108618861064800684FF47A71B0FBA4
:109AE000F1F0401E4FF0E021486107200861704707
:109AF0007C00002070B5F6F713FC0446102C16D33A
:109B000004F1E02090F8F05315480078854201DB1D
:109B1000012000E0002050B900BF502080F31188E0
:109B2000BFF34F8FBFF36F8F00BF00BFFEE70D483D
:109B3000006800F4E0600C490968884201D80120FF
:109B400000E0002050B900BF502080F31188BFF31F
:109B50004F8FBFF36F8F00BF00BFFEE770BD0000E7
:109B6000F80000200CED00E0FC0000200246002080
:109B70000BE0084B53F8303033B9064B43F8301044
:109B800003EBC0035A6002E0401C0828F1D300BF79
:109B9000704700006C2100202DE9F04105460E467B
:109BA00017462C46FFF7F8FE94F94400401C10B904
:109BB000002084F8440094F94500401C10B90020AE
:109BC00084F84500FFF712FFA06B28B93A463146EA
:109BD00004F1240000F0C6F82046FFF74DFDBDE873
:109BE000F081000070B504460025D4B11248006829
:109BF00008B9012000E0002050B900BF502080F3D8
:109C00001188BFF34F8FBFF36F8F00BF00BFFEE718
:109C100000F0AAF900212046FFF744F801F0F6F819
:109C200005463DB94FF0805004490860BFF34F8F9F
:109C3000BFF36F8F70BD0000B800002004ED00E09E
:109C400070B50546FFF7A8FE15B92748006800E083
:109C500028460446201DFFF727FEA06A18B104F12C
:109C60001800FFF721FE21480068401C1F490860CA
:109C70001D480068844209D1211D1D48FFF780FE60
:109C80001C480068401C1B49086009E01A4800682D
:109C9000401E194908602046FFF756F9FFF72EFCD1
:109CA000FFF7A4FE15480068E8B10F480068844239
:109CB00019D11348006808B9012000E0002050B90C
:109CC00000BF502080F31188BFF34F8FBFF36F8F19
:109CD00000BF00BFFEE74FF080500A490860BFF3A5
:109CE0004F8FBFF36F8F70BD80000020AC0000204D
:109CF000482600208C000020900000209C000020BE
:109D0000B800002004ED00E0034909680160034940
:109D10000968416070470000A800002094000020FE
:109D20000120014908607047A400002070B5044676
:109D30000D4654B900BF502080F31188BFF34F8FF8
:109D4000BFF36F8F00BF00BFFEE705480168183101
:109D50002046FFF7FBFD01212846FEF7A3FF70BD5B
:109D60008000002070B505460E46144655B900BF68
:109D7000502080F31188BFF34F8FBFF36F8F00BF68
:109D800000BFFEE70648016818312846FFF7F8FDD6
:109D90000CB14FF0FF3621463046FEF783FF70BD11
:109DA0008000002070B504460D46164654B900BF29
:109DB000502080F31188BFF34F8FBFF36F8F00BF28
:109DC00000BFFEE71048006808B1012000E0002055
:109DD00050B900BF502080F31188BFF34F8FBFF3FD
:109DE0006F8F00BF00BFFEE745F0004007490968DC
:109DF00088610648016818312046FFF7C1FD01213E
:109E00003046FEF74FFF70BDB800002080000020F4
:109E100070B505460E462148006808B1012000E0F3
:109E2000002050B900BF502080F31188BFF34F8F3E
:109E3000BFF36F8F00BF00BFFEE746F00040286011
:109E4000EC6854B900BF502080F31188BFF34F8FE6
:109E5000BFF36F8F00BF00BFFEE72846FFF724FD6A
:109E6000201DFFF721FD0E49E06A0968884202D9EA
:109E70000B49E06A0860E16A01EB8101094A02EBE3
:109E80008100211DFFF77CFD0749E06A0968C96A66
:109E9000884202D901200549086070BDB800002041
:109EA00098000020AC21002080000020A4000020A9
:109EB00010B586B000200590049003AA04A905A857
:109EC000FFF714FD0022DDE904101346CDE900215F
:109ED00002901EA11F48039A00F0DEFD1E49086093
:109EE0000846006808B1012400E00024012C02D1DA
:109EF00001F00EF80446012C15D100BF502080F36C
:109F00001188BFF34F8FBFF36F8F00BF4FF0FF304B
:109F100012490860012012490860002011490860B8
:109F200000F0A4F910E0601C08B1012000E000205E
:109F300050B900BF502080F31188BFF34F8FBFF39B
:109F40006F8F00BF00BFFEE706B010BD49444C450F
:109F5000000000003D900008B4000020B000002088
:109F60009C0000209400002002480068401C014929
:109F700008607047B80000201E48006818B1012032
:109F80001D49086034E000201B4908601B48016837
:109F90000CE051B900BF502080F31188BFF34F8F00
:109FA000BFF36F8F00BF00BFFEE7491E01EB8100CA
:109FB000134A52F8200008B9012000E000200028D0
:109FC000E7D101EB81020E4B03EB8200426852683D
:109FD000426000F108024368934202D1426852682D
:109FE00042604268D268074B1A600448016000BFB3
:109FF00070470000B8000020A40000209800002056
:10A00000AC2100208000002010B54FF0FF3300226B
:10A01000042102480068FEF7F9FC10BDB0010020E1
:10A020002DE9FE4F07468846002001903C460090EF
:10A0300057B900BF502080F31188BFF34F8FBFF393
:10A040006F8F00BF00BFFEE708F07F4008B9012016
:10A0500000E0002050B900BF502080F31188BFF30A
:10A060004F8FBFF36F8F00BF00BFFEE704F10409FD
:10A0700009F108000290FFF777FFD9F80C6020681B
:10A0800040EA0800206026E0D6F804B035680020D9
:10A09000009005F07F4A25F07F450AF0806028B9DE
:10A0A0002068284040B10120009005E02068284049
:10A0B000A84201D101200090009858B10AF08070A8
:10A0C00010B1019828430190206840F0007130469B
:10A0D000FFF79EFE5E4602988642D5D12068019920
:10A0E0008843206000F092FE2068BDE8FE8F0000EB
:10A0F0002DE9F04104460D46164633462A462146D0
:10A10000034800F083FF07463846BDE8F0810000B1
:10A110001D9900082DE9FF4F83B081460D46174673
:10A12000DDF840804C464FF0000A00200190B9F164
:10A13000000F0AD100BF502080F31188BFF34F8F6A
:10A14000BFF36F8F00BF00BFFEE705F07F4008B987
:10A15000012000E0002050B900BF502080F311889A
:10A16000BFF34F8FBFF36F8F00BF00BFFEE70DB18E
:10A17000012000E0002050B900BF502080F311887A
:10A18000BFF34F8FBFF36F8F00BF00BFFEE700F03C
:10A19000E7FC10B9B8F1000F01D1012000E0002068
:10A1A00050B900BF502080F31188BFF34F8FBFF329
:10A1B0006F8F00BF00BFFEE7FFF7D6FE206800905C
:10A1C0002946069A0098FFF73BFA0290029838B1A8
:10A1D000009E4FF00008C7B12068A843206014E03B
:10A1E000B8F1000F03D1009E012001900DE00FB1E6
:10A1F0004AF0807A069808B14AF0806A45EA0A0176
:10A200004246201DFFF7CEFD002600F0FFFD8346ED
:10A21000B8F1000F23D0BBF1000F07D14FF08050F1
:10A2200011490860BFF34F8FBFF36F8FFFF750FBEB
:10A23000064606F0007080B9FFF7AEFB2668294697
:10A240003046069AFFF7FCF918B117B12068A84309
:10A25000206001200190FFF7C9FB26F07F463046C1
:10A2600007B0BDE8F08F000004ED00E01CB55248D7
:10A2700000685249884201D0012000E0002050B916
:10A2800000BF502080F31188BFF34F8FBFF36F8F53
:10A2900000BF00BFFEE7484800684849491E8842A1
:10A2A00001D0012000E0002050B900BF502080F311
:10A2B0001188BFF34F8FBFF36F8F00BF00BFFEE762
:10A2C0003F49084600780190FF200A461070084672
:10A2D000007800909DF8000000F0F0009DF800204C
:10A2E000904201D1012000E0002050B900BF502071
:10A2F00080F31188BFF34F8FBFF36F8F00BF00BF94
:10A30000FEE79DF8000000F050002E4A1070072074
:10A310002D4A106009E02C480068401E2A4A10604F
:10A320009DF800004006000E00909DF8000000F02F
:10A3300080008028EFD024480068C0F1070004287E
:10A3400001D1012000E0002050B900BF502080F36F
:10A350001188BFF34F8FBFF36F8F00BF00BFFEE7C1
:10A36000194800680002184A10601046008800F47E
:10A37000E0601060124A019810700F4820300068A9
:10A3800040F470000C49203108600846006840F035
:10A3900070400860FFF79AFB00200C490860F5F751
:10A3A00087FF0B48006840F0404009490860F5F716
:10A3B0006BFF00201CBD000000ED00E071C20F41EA
:10A3C00000E400E0F8000020FC000020F400002081
:10A3D00034EF00E010B500BF502080F31188BFF3C8
:10A3E0004F8FBFF36F8F00BF00F0D0FB18B14FF05D
:10A3F00080500449086000BF002080F3118800BF2E
:10A4000010BD000004ED00E02DE9F84380460E4643
:10A4100017461D46DDF82090B8F1000F01D001204D
:10A4200000E0002050B900BF502080F31188BFF336
:10A430004F8FBFF36F8F00BF00BFFEE70DB101204C
:10A4400000E0002050B900BF502080F31188BFF316
:10A450004F8FBFF36F8F00BF00BFFEE707B10EB194
:10A46000012000E0002050B900BF502080F3118887
:10A47000BFF34F8FBFF36F8F00BF00BFFEE707B979
:10A480000EB9012000E0002050B900BF502080F339
:10A490001188BFF34F8FBFF36F8F00BF00BFFEE780
:10A4A000502000900098502801D1012000E00020A9
:10A4B00050B900BF502080F31188BFF34F8FBFF316
:10A4C0006F8F00BF00BFFEE700BF2C464CB10120DC
:10A4D00084F846004B463A46314640460094FEF723
:10A4E000C1FD2046BDE8F88370B505460E462C46F2
:10A4F00054B900BF502080F31188BFF34F8FBFF3D2
:10A500006F8F00BF00BFFEE7FFF746FAD4E90F12D6
:10A51000206801FB0200A0600020A063206860604A
:10A52000E06B401E226C216800FB0211E160FF20FD
:10A5300084F8440084F845009EB9206908B90120D8
:10A5400000E00020A8B904F1100000F013FC80B175
:10A550004FF0805009490860BFF34F8FBFF36F8FF2
:10A5600007E004F11000FFF7E1F904F12400FFF720
:10A57000DDF9FFF73BFA012070BD000004ED00E0BB
:10A580002DE9FF4383B0064688461D464FF000097B
:10A59000344654B900BF502080F31188BFF34F8F69
:10A5A000BFF36F8F00BF00BFFEE7B8F1000F01D10E
:10A5B000206C08B9012000E0002050B900BF5020F5
:10A5C00080F31188BFF34F8FBFF36F8F00BF00BFC1
:10A5D000FEE7022D02D1E06B012801D1012000E04D
:10A5E000002050B900BF502080F31188BFF34F8F77
:10A5F000BFF36F8F00BF00BFFEE700F0B1FA08B9EC
:10A60000059808B9012000E0002050B900BF502093
:10A6100080F31188BFF34F8FBFF36F8F00BF00BF70
:10A62000FEE700BFFFF7B8F9A06BE16B884201D3EA
:10A63000022D28D12A4641462046FEF746FC074611
:10A64000606A08B9012000E0002068B904F1240024
:10A6500000F090FB88B14FF0805032490860BFF3A2
:10A660004F8FBFF36F8F08E03FB14FF080502D49FF
:10A670000860BFF34F8FBFF36F8FFFF7B7F901206B
:10A6800007B0BDE8F083059818B9FFF7AFF90020CF
:10A69000F6E7B9F1000F04D101A8FFF735FB4FF041
:10A6A0000109FFF7A3F9FFF75FFCFFF775F994F9CC
:10A6B0004400401C10B9002084F8440094F945007F
:10A6C000401C10B9002084F84500FFF78FF905A958
:10A6D00001A800F05BF9F0B92046FEF7DAFDA0B161
:10A6E00004F110000599FFF721FB2046FEF7C4FF97
:10A6F00000F08CFB002895D14FF08050094908608C
:10A70000BFF34F8FBFF36F8F8CE72046FEF7B4FF88
:10A7100000F07CFB86E72046FEF7AEFF00F076FBFC
:10A720000020ADE704ED00E02DE9F84F07468A462A
:10A7300090461E463C4654B900BF502080F3118815
:10A74000BFF34F8FBFF36F8F00BF00BFFEE7BAF1BB
:10A75000000F01D1206C08B9012000E0002050B9A1
:10A7600000BF502080F31188BFF34F8FBFF36F8F6E
:10A7700000BF00BFFEE7022E02D1E06B012801D12D
:10A78000012000E0002050B900BF502080F3118864
:10A79000BFF34F8FBFF36F8F00BF00BFFEE7FFF720
:10A7A000A9F900BF5021EFF3118081F31188BFF3A5
:10A7B0004F8FBFF36F8F00BF0546A06BE16B8842E0
:10A7C00001D3022E25D194F945B0A06B00903246FA
:10A7D00051462046FEF779FB0BF1010088B9606A0B
:10A7E00008B9012000E0002050B904F1240000F075
:10A7F000C1FA28B1B8F1000F02D00120C8F800005A
:10A8000004E00BF1010040B284F845004FF001096B
:10A8100001E04FF0000900BF85F3118800BF4846F2
:10A82000BDE8F88F2DE9F74183B005460E464FF09D
:10A8300000082C4654B900BF502080F31188BFF3A4
:10A840004F8FBFF36F8F00BF00BFFEE70EB9206CC4
:10A8500008B9012000E0002050B900BF502080F36B
:10A860001188BFF34F8FBFF36F8F00BF00BFFEE7AC
:10A8700000F076F908B9059808B9012000E0002039
:10A8800050B900BF502080F31188BFF34F8FBFF342
:10A890006F8F00BF00BFFEE700BFFFF77DF8A76B1B
:10A8A000F7B131462046FEF7FBFA781EA063206917
:10A8B00008B9012000E0002060B904F1100000F0A8
:10A8C00059FA38B14FF080502F490860BFF34F8FCD
:10A8D000BFF36F8FFFF78AF8012006B0BDE8F08163
:10A8E000059818B9FFF782F80020F6E7B8F1000FD5
:10A8F00004D101A8FFF708FA4FF00108FFF776F836
:10A90000FFF732FBFFF748F894F94400401C10B9F8
:10A91000002084F8440094F94500401C10B9002040
:10A9200084F84500FFF762F805A901A800F02EF8A9
:10A93000F0B92046FEF7A0FCA0B104F1240005996F
:10A94000FFF7F4F92046FEF797FE00F05FFA0028C3
:10A95000A3D14FF080500C490860BFF34F8FBFF375
:10A960006F8F9AE72046FEF787FE00F04FFA94E7D4
:10A970002046FEF781FE00F049FA2046FEF77CFCF7
:10A9800000288AD00020A8E704ED00E070B5064654
:10A990000C4656B900BF502080F31188BFF34F8F8B
:10A9A000BFF36F8F00BF00BFFEE754B900BF502058
:10A9B00080F31188BFF34F8FBFF36F8F00BF00BFCD
:10A9C000FEE7FEF7E9FF184802687068131A174897
:10A9D000006890F85A0030B100201449096881F8E5
:10A9E0005A0001251CE02068401C08B9002517E02A
:10A9F0000F4930680968884204D07068904201D8D5
:10AA000001250DE02068984207D92068C01A20600F
:10AA10003046FFF779F9002502E00020206001258B
:10AA2000FEF7E4FF284670BD94000020800000205F
:10AA3000A80000202DE9FF4F85B0804689461746C3
:10AA4000DDE912ABB800FEF757FE064656B15C20B2
:10AA5000FEF752FE04460CB1266304E03046FEF7D2
:10AA6000E3FF00E000248CB1002084F85900CDE918
:10AA700000ABCDE902403A4649464046089BFEF706
:10AA800006FB2046FEF752F9012501E04FF0FF35A5
:10AA9000284609B0BDE8F08F2DE9F04F85B0074694
:10AAA000884691469A46DDE90EB6109C0EB101200B
:10AAB00000E0002050B900BF502080F31188BFF3A0
:10AAC0004F8FBFF36F8F00BF00BFFEE70CB10120B7
:10AAD00000E0002050B900BF502080F31188BFF380
:10AAE0004F8FBFF36F8F00BF00BFFEE75C20039066
:10AAF00003985C2801D1012000E0002050B900BF7C
:10AB0000502080F31188BFF34F8FBFF36F8F00BFCA
:10AB100000BFFEE700BFB4B1AEB125462C462E63A0
:10AB2000022085F85900002004A953464A46CDE981
:10AB300000B1CDE9025041463846FEF7A8FA284652
:10AB4000FEF7F4F801E000200490049805B0BDE899
:10AB5000F08F000001490868704700008000002065
:10AB60000549096809B9012005E00449096809B9DE
:10AB7000022000E0002070479C000020B800002068
:10AB80000149086870470000940000202DE9F04159
:10AB90004FF000084348006800287BD14248006815
:10ABA000451C4148056015BB40480068006808B96D
:10ABB000012000E0002050B900BF502080F3118830
:10ABC000BFF34F8FBFF36F8F00BF00BFFEE7374863
:10ABD00007683748006835490860354807603548D8
:10ABE0000068401C33490860FEF788FC00BF32480B
:10ABF000006885423BD300BF2C480068006808B954
:10AC0000012000E0002020B14FF0FF302A49086009
:10AC10002CE026480068C068C4686668B54202D265
:10AC20002548066022E0201DFEF73EFEA06A18B10E
:10AC300004F11800FEF738FE2049E06A09688842EE
:10AC400002D91E49E06A0860E16A01EB81011C4AF1
:10AC500002EB8100211DFEF793FE1A49E06A0968A4
:10AC6000C96A8842C8D34FF00108C5E700BF15483C
:10AC70000068C06A00EB8000114951F820000128EB
:10AC800001D94FF001081048006808B14FF00108E1
:10AC900005E0FFE70D480068401C0C49086040468D
:10ACA000BDE8F081B800002094000020840000205E
:10ACB00088000020A8000020B0000020980000209C
:10ACC000AC21002080000020A4000020A000002073
:10ACD00070B505462C460026002D43D0224800685A
:10ACE000844201D1012000E0002050B900BF502073
:10ACF00080F31188BFF34F8FBFF36F8F00BF00BF8A
:10AD0000FEE7206D50B900BF502080F31188BFF3DB
:10AD10004F8FBFF36F8F00BF00BFFEE7206D401E57
:10AD20002065E16CE06A88421CD0206DD0B9201DFE
:10AD3000FEF7BAFDE06CE062E06AC0F13800A061A5
:10AD40000A49E06A0968884202D90849E06A08604D
:10AD5000E16A01EB8101064A02EB8100211DFEF749
:10AD60000FFE0126304670BD8000002098000020B4
:10AD7000AC21002070B50646F068C46854B900BF25
:10AD8000502080F31188BFF34F8FBFF36F8F00BF48
:10AD900000BFFEE704F11800FEF786FD15480068C5
:10ADA000A0B9201DFEF780FD1349E06A09688842BA
:10ADB00002D91149E06A0860E16A01EB81010F4A9A
:10ADC00002EB8100211DFEF7DBFD04E004F1180118
:10ADD0000B48FEF7D5FD0B49E06A0968C96A88424D
:10ADE00004D9012501200849086000E00025284613
:10ADF00070BD0000B800002098000020AC210020A9
:10AE00003426002080000020A400002070B500241B
:10AE100000263648006850B900BF502080F31188E2
:10AE2000BFF34F8FBFF36F8F00BF00BFFEE7FEF78A
:10AE3000B3FD2E480068401E2C4908600846006893
:10AE400000284ED12A48006800284AD023E029482B
:10AE5000C068C46804F11800FEF726FD201DFEF747
:10AE600023FD2549E06A0968884202D92249E06A3F
:10AE70000860E16A01EB8101204A02EB8100211D9B
:10AE8000FEF77EFD1E49E06A0968C96A884202D35E
:10AE900001201C4908601748006808B9012000E03B
:10AEA00000200028D3D00CB1FEF728FB1648056817
:10AEB00065B100BFFFF76AFE10B1012011490860BB
:10AEC0006D1E002DF6D100200F4908600D48006866
:10AED00038B1012630070D490860BFF34F8FBFF32B
:10AEE0006F8FFEF783FD304670BD0000B800002074
:10AEF000900000203426002098000020AC21002083
:10AF000080000020A4000020A000002004ED00E04C
:10AF100010B586B00024FDF765FF16480068D0B173
:10AF200000200590049003AA04A905A8FEF7EAFCF6
:10AF30000222DDE904100023CDE9002102900EA1D8
:10AF40000F48039AFFF7A8FD0E49086008460068FD
:10AF500000B1012400BF54B900BF502080F3118814
:10AF6000BFF34F8FBFF36F8F00BF00BFFEE72046D8
:10AF700006B010BDC4000020546D722053766300EB
:10AF80005F960008C80000202DE9FF4704460D46E3
:10AF900016461F46DDF830804FF0000954B900BF57
:10AFA000502080F31188BFF34F8FBFF36F8F00BF26
:10AFB00000BFFEE71448006810B3009501960294A4
:10AFC000062D15DAFFF7CCFD022808D100234246F2
:10AFD00069460D480068FFF7D3FA814610E0002368
:10AFE0001A46694608480068FFF7CAFA814607E032
:10AFF00000233A46694604480068FFF795FB8146FE
:10B00000484604B0BDE8F087C40000202DE9FF41A8
:10B0100004460D4616461F466FF00100009001944D
:10B020000295039600233A46694604480068FFF7F4
:10B030007BFB8046404604B0BDE8F081C4000020A0
:10B040004FEA41034FEA5353A3F58063D3F11E0344
:10B05000C8BFD3F1210C0CDD4FF0004242EAC122FF
:10B0600042EA505232FA03FC8CEAE17CACEBE1702C
:10B070007047102BC4BF0020704703F5787CBCF1EB
:10B08000FF3F04D06FF0004282EA2100704770B5A4
:10B0900000F0C6F84992248000207047F2E710F0D3
:10B0A000004248BF4042B0FA80F310FA03F10AD0E0
:10B0B000C3F11D0303F580634FEA415002EB0352D5
:10B0C00002EBD12170474FF000007047DFF848C114
:10B0D00070B51CEA111E1EBF1CEA13159EEA0C0F68
:10B0E00095EA0C0F00F06F8081EA030423EA4C1309
:10B0F0004EEAD47E21EA4C1141F4801143F48013CE
:10B10000AE44A1FB024CA0FB0365AEF17F7E361975
:10B1100055EB0C05A1FB034C4CF10003A0FB021CFA
:10B1200016EB0C06654153F10003094218BF46F0C7
:10B13000010613F4007F0BD14FEA03314FEA0530CB
:10B14000340341EA155140EA16506FF003020AE059
:10B150004FEAC3214FEAC520F40241EA555140EAC3
:10B1600056506FF0020202EB2E4201EB025585EAC7
:10B17000CE710AD05FEA440C18BF24F0004450F1AD
:10B18000000041F1000120EAD47040F2FE7C6245EB
:10B1900000D270BDA84214BF4FF080444FF040442D
:10B1A000002E08BF0024BEF1806FA8BFA1F1C041EE
:10B1B000BDE8704080F282804FF0000001F1C04194
:10B1C00001F0004170479EEA0C0F0CEA131518BFFE
:10B1D00095EA0C0F06D04FF0000081EA030E0EF046
:10B1E000004170BD00F01CF88900013E00F007B876
:10B1F00000F009B84FEA430C5FEA5C5C08D081EAD2
:10B20000030100F05BB84FEA410C5FEA5C5CF6D1E9
:10B210004FF00000014970470000FF070000F87F71
:10B220000EF1020E2EF0030E5EF8046B364205D4CA
:10B23000012A43EB030515F5001F12D8012841EB45
:10B24000010C1CF5001F0CD80ED14FEAD17C15F56E
:10B25000001F0CEB4C0C0CF1020C08BF4CEBD37C28
:10B2600004E04FF0080C01E04FEAD37C0CEB4C05F6
:10B2700026FA05F606F00706B6F1040C06D20EEB28
:10B28000860CBDE870404CF0010C6047DFE80CF024
:10B29000090B02024FF000414FF00000A1F5002120
:10B2A00070BD19461046012851EB010418BFD4F5B2
:10B2B000001484BF002001F0004170BD0808A0F513
:10B2C00000114FEA310170474FF04070E1EE100A73
:10B2D0007047000080B80008000000000000000077
:10B2E0000000000000000000000200001800000044
:10B2F00000000000000000000006101600061016F6
:10B300000000000000000000010203040607080915
:10B310000000000001020304000000008911000089
:10B32000122300009B32000024460000AD570000AD
:10B3300036650000BF740000488C0000C19D00000D
:10B340005AAF0000D3BE00006CCA0000E5DB00006D
:10B350007EE90000F7F800008110000008010000FD
:10B36000933300001A220000A55600002C4700006D
:10B37000B77500003E640000C99C0000408D0000CD
:10B38000DBBF000052AE0000EDDA000064CB00002D
:10B39000FFF9000076E80000022100008B30000079
:10B3A000100200009913000026670000AF7600002D
:10B3B00034440000BD5500004AAD0000C3BC00008D
:10B3C000588E0000D19F00006EEB0000E7FA0000ED
:10B3D0007CC80000F5D90000833100000A2000007D
:10B3E0009112000018030000A77700002E660000ED
:10B3F000B55400003C450000CBBD000042AC00004D
:10B40000D99E0000508F0000EFFB000066EA0000AC
:10B41000FDD8000074C90000044200008D530000F4
:10B42000166100009F70000020040000A9150000B4
:10B4300032270000BB3600004CCE0000C5DF000004
:10B440005EED0000D7FC000068880000E199000074
:10B450007AAB0000F3BA0000855200000C430000F4
:10B46000977100001E600000A11400002805000074
:10B47000B33700003A260000CDDE000044CF0000C4
:10B48000DFFD000056EC0000E99800006089000034
:10B49000FBBB000072AA0000066300008F72000070
:10B4A000144000009D51000022250000AB34000034
:10B4B00030060000B91700004EEF0000C7FE000084
:10B4C0005CCC0000D5DD00006AA90000E3B80000F4
:10B4D000788A0000F19B0000877300000E62000074
:10B4E000955000001C410000A33500002A240000F4
:10B4F000B116000038070000CFFF000046EE000044
:10B50000DDDC000054CD0000EBB9000062A80000B3
:10B51000F99A0000708B00000884000081950000FB
:10B520001AA7000093B600002CC20000A5D30000AB
:10B530003EE10000B7F0000040080000C91900001B
:10B54000522B0000DB3A0000644E0000ED5F00006B
:10B55000766D0000FF7C00008994000000850000EB
:10B560009BB7000012A60000ADD2000024C300006B
:10B57000BFF1000036E00000C118000048090000DB
:10B58000D33B00005A2A0000E55E00006C4F00002B
:10B59000F77D00007E6C00000AA5000083B4000067
:10B5A00018860000919700002EE30000A7F200002B
:10B5B0003CC00000B5D1000042290000CB3800009B
:10B5C000500A0000D91B0000666F0000EF7E0000EB
:10B5D000744C0000FD5D00008BB5000002A400006B
:10B5E0009996000010870000AFF3000026E20000EB
:10B5F000BDD0000034C10000C33900004A2800005B
:10B60000D11A0000580B0000E77F00006E6E0000AA
:10B61000F55C00007C4D00000CC6000085D70000E2
:10B620001EE5000097F4000028800000A1910000B2
:10B630003AA30000B3B20000444A0000CD5B000012
:10B6400056690000DF780000600C0000E91D000072
:10B65000722F0000FB3E00008DD6000004C70000E2
:10B660009FF5000016E40000A99000002081000072
:10B67000BBB3000032A20000C55A00004C4B0000D2
:10B68000D77900005E680000E11C0000680D000032
:10B69000F33F00007A2E00000EE7000087F600005E
:10B6A0001CC4000095D500002AA10000A3B0000032
:10B6B00038820000B1930000466B0000CF7A000092
:10B6C00054480000DD590000622D0000EB3C0000F2
:10B6D000700E0000F91F00008FF7000006E6000062
:10B6E0009DD4000014C50000ABB1000022A00000F2
:10B6F000B992000030830000C77B00004E6A000052
:10B70000D55800005C490000E33D00006A2C0000B1
:10B71000F11E0000780F0000D8B8000800000000FB
:10B720000000000000000000000000000004000015
:10B7300030000000000000000000000098B8000881
:10B7400000000000000000000000000000000000F9
:10B7500000020000300000000000000000000000B7
:10B76000B8B8000800000000000000000000000061
:10B770000000000000020000300000000000000097
:10B7800000000000C0B80008000000000000000039
:10B790000000000000000000000200003000000077
:10B7A0000000000000000000E0B8000800000000F9
:10B7B0000000000000000000000000000004000085
:10B7C000300000000000000000000000BCB80008CD
:10B7D0000000000000000000000000000000000069
:10B7E0000004000030000000000000000000000025
:10B7F000C8B80008000000000000000000000000C1
:10B800000000000000040000300000000000000004
:10B81000000000009CB800080000000000000000CC
:10B8200000000000000000000004000030000000E4
:10B830000000000000000000A8B8000800000000A0
:10B8400000000000000000000000000000040000F4
:10B850003000000000000000000000008CB800086C
:10B8600000000000000000000000000000000000D8
:10B870000004000030000000000000000000000094
:10B88000696E69745461736B0000000067696D62D2
:10B89000616C5F72656300006C6564006C65667462
:10B8A0005F67696D62616C0072696768745F676980
:10B8B0006D62616C0000000063616E00676F0000E4
:10B8C0006D6F746F720000006374726C5F63686107
:10B8D0007373697300000000696E697400000000F2
:10B8E00073686F6F7400000008B900080000002042
:10B8F0000C020000C4010008E0B900080C0200209E
:10B900005C74000020020008C113C56014080D61BA
:10B910001B081D041A49041A89041A91141AD50423
:10B92000131201140202021640830440572602013A
:10B93000020301071A040309041A0313B5071B08BD
:10B94000B1041A6D041AD9041AF504413210193FD2
:10B9500021037524F41AAA01C1130A0632022A40EF
:10B96000941BD95BF012594C08235EAC13A95A14EE
:10B9700008C9581B088D14C11A4D281A09041A95B4
:10B98000041AF924140902431302011DC0320904E8
:10B99000DD1A020B130524161001052401100901FC
:10B9A0000424020205240617010705820308151066
:10B9B00009040133020A2E0705010240072A810704
:10B9C000044C81018267A0409A99993E63C841A0C6
:10B9D0000BC03FCDCC9C400AD7233C74204164006F
:040000050800018965
:00000001FF
